MPLINK 4.35, Linker
Linker Map File - Created Sat Oct 23 17:06:12 2010

                                 Section Info
                  Section       Type    Address   Location Size(Bytes)
                ---------  ---------  ---------  ---------  ---------
               _entry_scn       code   0x000000    program   0x000006
    HIGH_INTERRUPT_VECTOR       code   0x000008    program   0x000006
     LOW_INTERRUPT_VECTOR       code   0x000018    program   0x000006
    REMAPPED_RESET_VECTOR       code   0x001000    program   0x000006
REMAPPED_HIGH_INTERRUPT_VECTOR       code   0x001008    program   0x000006
REMAPPED_LOW_INTERRUPT_VECTOR       code   0x001018    program   0x000006
                   .cinit    romdata   0x00102a    program   0x00001a
         .code_MainDemo.o       code   0x001044    program   0x00027e
        .code_TimeDelay.o       code   0x0012c2    program   0x000224
               _cinit_scn       code   0x0014e6    program   0x00009e
          .code_fxm3232.o       code   0x001584    program   0x000070
             .code_tick.o       code   0x0015f4    program   0x00003a
                    .code       code   0x00162e    program   0x000020
             _startup_scn       code   0x00164e    program   0x00001c
           .code___init.o       code   0x00166a    program   0x000002
     .romdata_TimeDelay.o    romdata   0x00166c    program   0x000000
          .romdata_tick.o    romdata   0x00166c    program   0x000000
          .idata_tick.o_i    romdata   0x00166c    program   0x000004
       .romdata_fxm3232.o    romdata   0x00166c    program   0x000000
         .romdata_c018i.o    romdata   0x00166c    program   0x000000
      .romdata_MainDemo.o    romdata   0x00166c    program   0x000000
        .romdata___init.o    romdata   0x00166c    program   0x000000
       .idata_fxm3232.o_i    romdata   0x001670    program   0x000000
        .idata___init.o_i    romdata   0x001670    program   0x000000
     .idata_TimeDelay.o_i    romdata   0x001670    program   0x000000
      .idata_MainDemo.o_i    romdata   0x001670    program   0x000006
         .idata_c018i.o_i    romdata   0x001670    program   0x000000
            .code_c018i.o       code   0x001676    program   0x000000
 .config_1fff8_MainDemo.o    romdata   0x01fff8    program   0x000001
 .config_1fff9_MainDemo.o    romdata   0x01fff9    program   0x000001
 .config_1fffa_MainDemo.o    romdata   0x01fffa    program   0x000001
 .config_1fffb_MainDemo.o    romdata   0x01fffb    program   0x000001
 .config_1fffd_MainDemo.o    romdata   0x01fffd    program   0x000001
                MATH_DATA      udata   0x000000       data   0x000010
                 .tmpdata      udata   0x000010       data   0x000004
                   .stack      udata   0x000e00       data   0x000100
           .udata_c018i.o      udata   0x000f00       data   0x00000a
        .udata_MainDemo.o      udata   0x000f0a       data   0x000008
        .idata_MainDemo.o      idata   0x000f12       data   0x000006
            .idata_tick.o      idata   0x000f18       data   0x000004
           .idata_c018i.o      idata   0x000f1c       data   0x000000
            .udata_tick.o      udata   0x000f1c       data   0x000000
       .udata_TimeDelay.o      udata   0x000f1c       data   0x000000
       .idata_TimeDelay.o      idata   0x000f1c       data   0x000000
         .udata_fxm3232.o      udata   0x000f1c       data   0x000000
         .idata_fxm3232.o      idata   0x000f1c       data   0x000000
          .udata___init.o      udata   0x000f1c       data   0x000000
          .idata___init.o      idata   0x000f1c       data   0x000000
              SFR_BANKED0      udata   0x000f40       data   0x000020
            SFR_UNBANKED0      udata   0x000f60       data   0x0000a0



                              Program Memory Usage 
                               Start         End      
                           ---------   ---------      
                            0x000000    0x000005      
                            0x000008    0x00000d      
                            0x000018    0x00001d      
                            0x001000    0x001005      
                            0x001008    0x00100d      
                            0x001018    0x00101d      
                            0x00102a    0x001675      
                            0x01fff8    0x01fffb      
                            0x01fffd    0x01fffd      
            1653 out of 131072 program addresses used, program memory utilization is 1%



                              Symbols - Sorted by Name
                     Name    Address   Location    Storage File                     
                ---------  ---------  ---------  --------- ---------                
                Delay10us   0x0012c2    program     extern D:\Projects\PIC18_USB_Eval\Firmware\SoftPowerOnOff\TimeDelay\TimeDelay.c
                  DelayMs   0x0013d8    program     extern D:\Projects\PIC18_USB_Eval\Firmware\SoftPowerOnOff\TimeDelay\TimeDelay.c
                  FXM3232   0x001584    program     extern C:\MCC18\src\traditional\math\fxm3232.c
                 High_ISR   0x000008    program     extern D:\Projects\PIC18_USB_Eval\Firmware\SoftPowerOnOff\SoftPowerOnOff\MainDemo.c
                  Low_ISR   0x000018    program     extern D:\Projects\PIC18_USB_Eval\Firmware\SoftPowerOnOff\SoftPowerOnOff\MainDemo.c
        Remapped_High_ISR   0x001008    program     extern D:\Projects\PIC18_USB_Eval\Firmware\SoftPowerOnOff\SoftPowerOnOff\MainDemo.c
         Remapped_Low_ISR   0x001018    program     extern D:\Projects\PIC18_USB_Eval\Firmware\SoftPowerOnOff\SoftPowerOnOff\MainDemo.c
                  TickGet   0x001606    program     extern D:\Projects\PIC18_USB_Eval\Firmware\SoftPowerOnOff\Tick\tick.c
                 TickInit   0x0015f4    program     extern D:\Projects\PIC18_USB_Eval\Firmware\SoftPowerOnOff\Tick\tick.c
               TickUpdate   0x001618    program     extern D:\Projects\PIC18_USB_Eval\Firmware\SoftPowerOnOff\Tick\tick.c
  YourHighPriorityISRCode   0x001044    program     extern D:\Projects\PIC18_USB_Eval\Firmware\SoftPowerOnOff\SoftPowerOnOff\MainDemo.c
   YourLowPriorityISRCode   0x001110    program     extern D:\Projects\PIC18_USB_Eval\Firmware\SoftPowerOnOff\SoftPowerOnOff\MainDemo.c
           ___?:_lbl00026   0x00120e    program     static                          
           ___?:_lbl00027   0x001208    program     static                          
       ___case_0_lbl00019   0x0011b2    program     static                          
       ___case_1_lbl00022   0x0011c2    program     static                          
       ___case_2_lbl00025   0x0011d4    program     static                          
         ___else_lbl00004   0x001378    program     static                          
         ___else_lbl00006   0x0012d2    program     static                          
         ___else_lbl00011   0x001486    program     static                          
         ___else_lbl00021   0x0011ce    program     static                          
         ___else_lbl00024   0x0011de    program     static                          
         ___else_lbl00033   0x00121a    program     static                          
         ___else_lbl00038   0x001252    program     static                          
           ___if_lbl00003   0x0013c4    program     static                          
           ___if_lbl00005   0x0013c4    program     static                          
           ___if_lbl00010   0x0014d2    program     static                          
           ___if_lbl00016   0x00116a    program     static                          
           ___if_lbl00018   0x0011c0    program     static                          
           ___if_lbl00020   0x0011d2    program     static                          
           ___if_lbl00023   0x0011e4    program     static                          
           ___if_lbl00028   0x001218    program     static                          
           ___if_lbl00029   0x001218    program     static                          
           ___if_lbl00030   0x00122c    program     static                          
           ___if_lbl00031   0x001234    program     static                          
           ___if_lbl00032   0x001234    program     static                          
           ___if_lbl00034   0x001234    program     static                          
           ___if_lbl00037   0x001256    program     static                          
           ___if_lbl00039   0x00126a    program     static                          
       ___return_lbl00000   0x001004    program     static                          
       ___return_lbl00000   0x0013c4    program     static                          
       ___return_lbl00000   0x000004    program     static                          
       ___return_lbl00000   0x0015f2    program     static                          
       ___return_lbl00001   0x001668    program     static                          
       ___return_lbl00001   0x00100c    program     static                          
       ___return_lbl00002   0x00101c    program     static                          
       ___return_lbl00002   0x001582    program     static                          
       ___return_lbl00003   0x00000c    program     static                          
       ___return_lbl00004   0x00001c    program     static                          
       ___return_lbl00007   0x0014d2    program     static                          
       ___return_lbl00015   0x00126a    program     static                          
   ___switchexit_lbl00017   0x0011e4    program     static                          
        ___while_lbl00001   0x001378    program     static                          
        ___while_lbl00002   0x0013c4    program     static                          
        ___while_lbl00008   0x001486    program     static                          
        ___while_lbl00009   0x0014d2    program     static                          
               __config_0   0x01fff8    program     static D:\Projects\PIC18_USB_Eval\Firmware\SoftPowerOnOff\SoftPowerOnOff\MainDemo.c
               __config_1   0x01fff9    program     static D:\Projects\PIC18_USB_Eval\Firmware\SoftPowerOnOff\SoftPowerOnOff\MainDemo.c
               __config_2   0x01fffa    program     static D:\Projects\PIC18_USB_Eval\Firmware\SoftPowerOnOff\SoftPowerOnOff\MainDemo.c
               __config_3   0x01fffb    program     static D:\Projects\PIC18_USB_Eval\Firmware\SoftPowerOnOff\SoftPowerOnOff\MainDemo.c
               __config_4   0x01fffd    program     static D:\Projects\PIC18_USB_Eval\Firmware\SoftPowerOnOff\SoftPowerOnOff\MainDemo.c
                   __init   0x00166a    program     extern C:\MCC18\src\traditional\stdclib\__init.c
               __tmplbl_0   0x001374    program     static                          
               __tmplbl_0   0x00119e    program     static                          
               __tmplbl_1   0x00124a    program     static                          
               __tmplbl_1   0x0013a6    program     static                          
               __tmplbl_2   0x00123c    program     static                          
               __tmplbl_2   0x001480    program     static                          
               __tmplbl_3   0x001242    program     static                          
               __tmplbl_3   0x0014b4    program     static                          
            __zero_memory   0x00162e    program     extern C:\MCC18\src\traditional\proc\p18F67J50.asm
                _do_cinit   0x0014e6    program     extern C:\MCC18\src\traditional\startup\c018i.c
                   _entry   0x000000    program     extern C:\MCC18\src\traditional\startup\c018i.c
                   _reset   0x001000    program     extern D:\Projects\PIC18_USB_Eval\Firmware\SoftPowerOnOff\SoftPowerOnOff\MainDemo.c
                 _startup   0x00164e    program     extern C:\MCC18\src\traditional\startup\c018i.c
                compare_l   0x001644    program     static C:\MCC18\src\traditional\proc\p18F67J50.asm
                copy_loop   0x001558    program     static                          
            copy_one_byte   0x00155e    program     static                          
                     done   0x001582    program     static                          
             done_copying   0x00156c    program     static                          
                  ledTask   0x00126c    program     extern D:\Projects\PIC18_USB_Eval\Firmware\SoftPowerOnOff\SoftPowerOnOff\MainDemo.c
                     loop   0x00165e    program     static                          
                   loop_h   0x00163c    program     static C:\MCC18\src\traditional\proc\p18F67J50.asm
                   loop_l   0x001646    program     static C:\MCC18\src\traditional\proc\p18F67J50.asm
                     main   0x001136    program     extern D:\Projects\PIC18_USB_Eval\Firmware\SoftPowerOnOff\SoftPowerOnOff\MainDemo.c
                     test   0x001500    program     static                          
                   uiTask   0x00115a    program     extern D:\Projects\PIC18_USB_Eval\Firmware\SoftPowerOnOff\SoftPowerOnOff\MainDemo.c
               zero_block   0x00163c    program     static C:\MCC18\src\traditional\proc\p18F67J50.asm
                   ADCON0   0x000fc2       data     extern C:\MCC18\src\traditional\proc\p18F67J50.asm
               ADCON0bits   0x000fc2       data     extern C:\MCC18\src\traditional\proc\p18F67J50.asm
                   ADCON1   0x000fc1       data     extern C:\MCC18\src\traditional\proc\p18F67J50.asm
               ADCON1bits   0x000fc1       data     extern C:\MCC18\src\traditional\proc\p18F67J50.asm
                    ADRES   0x000fc3       data     extern C:\MCC18\src\traditional\proc\p18F67J50.asm
                   ADRESH   0x000fc4       data     extern C:\MCC18\src\traditional\proc\p18F67J50.asm
                   ADRESL   0x000fc3       data     extern C:\MCC18\src\traditional\proc\p18F67J50.asm
                   ANCON0   0x000fc1       data     extern C:\MCC18\src\traditional\proc\p18F67J50.asm
               ANCON0bits   0x000fc1       data     extern C:\MCC18\src\traditional\proc\p18F67J50.asm
                   ANCON1   0x000fc2       data     extern C:\MCC18\src\traditional\proc\p18F67J50.asm
               ANCON1bits   0x000fc2       data     extern C:\MCC18\src\traditional\proc\p18F67J50.asm
                  BAUDCON   0x000f7e       data     extern C:\MCC18\src\traditional\proc\p18F67J50.asm
                 BAUDCON1   0x000f7e       data     extern C:\MCC18\src\traditional\proc\p18F67J50.asm
             BAUDCON1bits   0x000f7e       data     extern C:\MCC18\src\traditional\proc\p18F67J50.asm
                 BAUDCON2   0x000f7c       data     extern C:\MCC18\src\traditional\proc\p18F67J50.asm
             BAUDCON2bits   0x000f7c       data     extern C:\MCC18\src\traditional\proc\p18F67J50.asm
              BAUDCONbits   0x000f7e       data     extern C:\MCC18\src\traditional\proc\p18F67J50.asm
                      BSR   0x000fe0       data     extern C:\MCC18\src\traditional\proc\p18F67J50.asm
                  CCP1CON   0x000fbb       data     extern C:\MCC18\src\traditional\proc\p18F67J50.asm
              CCP1CONbits   0x000fbb       data     extern C:\MCC18\src\traditional\proc\p18F67J50.asm
                  CCP2CON   0x000fb6       data     extern C:\MCC18\src\traditional\proc\p18F67J50.asm
              CCP2CONbits   0x000fb6       data     extern C:\MCC18\src\traditional\proc\p18F67J50.asm
                  CCP3CON   0x000fb1       data     extern C:\MCC18\src\traditional\proc\p18F67J50.asm
              CCP3CONbits   0x000fb1       data     extern C:\MCC18\src\traditional\proc\p18F67J50.asm
                  CCP4CON   0x000f73       data     extern C:\MCC18\src\traditional\proc\p18F67J50.asm
              CCP4CONbits   0x000f73       data     extern C:\MCC18\src\traditional\proc\p18F67J50.asm
                  CCP5CON   0x000f70       data     extern C:\MCC18\src\traditional\proc\p18F67J50.asm
              CCP5CONbits   0x000f70       data     extern C:\MCC18\src\traditional\proc\p18F67J50.asm
                    CCPR1   0x000fbc       data     extern C:\MCC18\src\traditional\proc\p18F67J50.asm
                   CCPR1H   0x000fbd       data     extern C:\MCC18\src\traditional\proc\p18F67J50.asm
                   CCPR1L   0x000fbc       data     extern C:\MCC18\src\traditional\proc\p18F67J50.asm
                    CCPR2   0x000fb7       data     extern C:\MCC18\src\traditional\proc\p18F67J50.asm
                   CCPR2H   0x000fb8       data     extern C:\MCC18\src\traditional\proc\p18F67J50.asm
                   CCPR2L   0x000fb7       data     extern C:\MCC18\src\traditional\proc\p18F67J50.asm
                    CCPR3   0x000fb2       data     extern C:\MCC18\src\traditional\proc\p18F67J50.asm
                   CCPR3H   0x000fb3       data     extern C:\MCC18\src\traditional\proc\p18F67J50.asm
                   CCPR3L   0x000fb2       data     extern C:\MCC18\src\traditional\proc\p18F67J50.asm
                    CCPR4   0x000f74       data     extern C:\MCC18\src\traditional\proc\p18F67J50.asm
                   CCPR4H   0x000f75       data     extern C:\MCC18\src\traditional\proc\p18F67J50.asm
                   CCPR4L   0x000f74       data     extern C:\MCC18\src\traditional\proc\p18F67J50.asm
                    CCPR5   0x000f71       data     extern C:\MCC18\src\traditional\proc\p18F67J50.asm
                   CCPR5H   0x000f72       data     extern C:\MCC18\src\traditional\proc\p18F67J50.asm
                   CCPR5L   0x000f71       data     extern C:\MCC18\src\traditional\proc\p18F67J50.asm
                   CM1CON   0x000fd2       data     extern C:\MCC18\src\traditional\proc\p18F67J50.asm
                  CM1CON1   0x000fd2       data     extern C:\MCC18\src\traditional\proc\p18F67J50.asm
              CM1CON1bits   0x000fd2       data     extern C:\MCC18\src\traditional\proc\p18F67J50.asm
               CM1CONbits   0x000fd2       data     extern C:\MCC18\src\traditional\proc\p18F67J50.asm
                   CM2CON   0x000fd1       data     extern C:\MCC18\src\traditional\proc\p18F67J50.asm
                  CM2CON1   0x000fd1       data     extern C:\MCC18\src\traditional\proc\p18F67J50.asm
              CM2CON1bits   0x000fd1       data     extern C:\MCC18\src\traditional\proc\p18F67J50.asm
               CM2CONbits   0x000fd1       data     extern C:\MCC18\src\traditional\proc\p18F67J50.asm
                   CMSTAT   0x000f6a       data     extern C:\MCC18\src\traditional\proc\p18F67J50.asm
                 CMSTATUS   0x000f6a       data     extern C:\MCC18\src\traditional\proc\p18F67J50.asm
             CMSTATUSbits   0x000f6a       data     extern C:\MCC18\src\traditional\proc\p18F67J50.asm
               CMSTATbits   0x000f6a       data     extern C:\MCC18\src\traditional\proc\p18F67J50.asm
                   CVRCON   0x000f77       data     extern C:\MCC18\src\traditional\proc\p18F67J50.asm
               CVRCONbits   0x000f77       data     extern C:\MCC18\src\traditional\proc\p18F67J50.asm
                     DDRA   0x000f92       data     extern C:\MCC18\src\traditional\proc\p18F67J50.asm
                 DDRAbits   0x000f92       data     extern C:\MCC18\src\traditional\proc\p18F67J50.asm
                     DDRB   0x000f93       data     extern C:\MCC18\src\traditional\proc\p18F67J50.asm
                 DDRBbits   0x000f93       data     extern C:\MCC18\src\traditional\proc\p18F67J50.asm
                     DDRC   0x000f94       data     extern C:\MCC18\src\traditional\proc\p18F67J50.asm
                 DDRCbits   0x000f94       data     extern C:\MCC18\src\traditional\proc\p18F67J50.asm
                     DDRD   0x000f95       data     extern C:\MCC18\src\traditional\proc\p18F67J50.asm
                 DDRDbits   0x000f95       data     extern C:\MCC18\src\traditional\proc\p18F67J50.asm
                     DDRE   0x000f96       data     extern C:\MCC18\src\traditional\proc\p18F67J50.asm
                 DDREbits   0x000f96       data     extern C:\MCC18\src\traditional\proc\p18F67J50.asm
                     DDRF   0x000f97       data     extern C:\MCC18\src\traditional\proc\p18F67J50.asm
                 DDRFbits   0x000f97       data     extern C:\MCC18\src\traditional\proc\p18F67J50.asm
                     DDRG   0x000f98       data     extern C:\MCC18\src\traditional\proc\p18F67J50.asm
                 DDRGbits   0x000f98       data     extern C:\MCC18\src\traditional\proc\p18F67J50.asm
                  ECCP1AS   0x000fbf       data     extern C:\MCC18\src\traditional\proc\p18F67J50.asm
              ECCP1ASbits   0x000fbf       data     extern C:\MCC18\src\traditional\proc\p18F67J50.asm
                 ECCP1CON   0x000fbb       data     extern C:\MCC18\src\traditional\proc\p18F67J50.asm
             ECCP1CONbits   0x000fbb       data     extern C:\MCC18\src\traditional\proc\p18F67J50.asm
                 ECCP1DEL   0x000fbe       data     extern C:\MCC18\src\traditional\proc\p18F67J50.asm
             ECCP1DELbits   0x000fbe       data     extern C:\MCC18\src\traditional\proc\p18F67J50.asm
                  ECCP2AS   0x000fba       data     extern C:\MCC18\src\traditional\proc\p18F67J50.asm
              ECCP2ASbits   0x000fba       data     extern C:\MCC18\src\traditional\proc\p18F67J50.asm
                 ECCP2CON   0x000fb6       data     extern C:\MCC18\src\traditional\proc\p18F67J50.asm
             ECCP2CONbits   0x000fb6       data     extern C:\MCC18\src\traditional\proc\p18F67J50.asm
                 ECCP2DEL   0x000fb9       data     extern C:\MCC18\src\traditional\proc\p18F67J50.asm
             ECCP2DELbits   0x000fb9       data     extern C:\MCC18\src\traditional\proc\p18F67J50.asm
                  ECCP3AS   0x000fb5       data     extern C:\MCC18\src\traditional\proc\p18F67J50.asm
              ECCP3ASbits   0x000fb5       data     extern C:\MCC18\src\traditional\proc\p18F67J50.asm
                 ECCP3CON   0x000fb1       data     extern C:\MCC18\src\traditional\proc\p18F67J50.asm
             ECCP3CONbits   0x000fb1       data     extern C:\MCC18\src\traditional\proc\p18F67J50.asm
                 ECCP3DEL   0x000fb4       data     extern C:\MCC18\src\traditional\proc\p18F67J50.asm
             ECCP3DELbits   0x000fb4       data     extern C:\MCC18\src\traditional\proc\p18F67J50.asm
                   EECON1   0x000fa6       data     extern C:\MCC18\src\traditional\proc\p18F67J50.asm
               EECON1bits   0x000fa6       data     extern C:\MCC18\src\traditional\proc\p18F67J50.asm
                   EECON2   0x000fa7       data     extern C:\MCC18\src\traditional\proc\p18F67J50.asm
                     FSR0   0x000fe9       data     extern C:\MCC18\src\traditional\proc\p18F67J50.asm
                    FSR0H   0x000fea       data     extern C:\MCC18\src\traditional\proc\p18F67J50.asm
                    FSR0L   0x000fe9       data     extern C:\MCC18\src\traditional\proc\p18F67J50.asm
                     FSR1   0x000fe1       data     extern C:\MCC18\src\traditional\proc\p18F67J50.asm
                    FSR1H   0x000fe2       data     extern C:\MCC18\src\traditional\proc\p18F67J50.asm
                    FSR1L   0x000fe1       data     extern C:\MCC18\src\traditional\proc\p18F67J50.asm
                     FSR2   0x000fd9       data     extern C:\MCC18\src\traditional\proc\p18F67J50.asm
                    FSR2H   0x000fda       data     extern C:\MCC18\src\traditional\proc\p18F67J50.asm
                    FSR2L   0x000fd9       data     extern C:\MCC18\src\traditional\proc\p18F67J50.asm
                    INDF0   0x000fef       data     extern C:\MCC18\src\traditional\proc\p18F67J50.asm
                    INDF1   0x000fe7       data     extern C:\MCC18\src\traditional\proc\p18F67J50.asm
                    INDF2   0x000fdf       data     extern C:\MCC18\src\traditional\proc\p18F67J50.asm
                   INTCON   0x000ff2       data     extern C:\MCC18\src\traditional\proc\p18F67J50.asm
                  INTCON2   0x000ff1       data     extern C:\MCC18\src\traditional\proc\p18F67J50.asm
              INTCON2bits   0x000ff1       data     extern C:\MCC18\src\traditional\proc\p18F67J50.asm
                  INTCON3   0x000ff0       data     extern C:\MCC18\src\traditional\proc\p18F67J50.asm
              INTCON3bits   0x000ff0       data     extern C:\MCC18\src\traditional\proc\p18F67J50.asm
               INTCONbits   0x000ff2       data     extern C:\MCC18\src\traditional\proc\p18F67J50.asm
                     IPR1   0x000f9f       data     extern C:\MCC18\src\traditional\proc\p18F67J50.asm
                 IPR1bits   0x000f9f       data     extern C:\MCC18\src\traditional\proc\p18F67J50.asm
                     IPR2   0x000fa2       data     extern C:\MCC18\src\traditional\proc\p18F67J50.asm
                 IPR2bits   0x000fa2       data     extern C:\MCC18\src\traditional\proc\p18F67J50.asm
                     IPR3   0x000fa5       data     extern C:\MCC18\src\traditional\proc\p18F67J50.asm
                 IPR3bits   0x000fa5       data     extern C:\MCC18\src\traditional\proc\p18F67J50.asm
               KeyDownTmr   0x000f16       data     extern D:\Projects\PIC18_USB_Eval\Firmware\SoftPowerOnOff\SoftPowerOnOff\MainDemo.c
                KeyHitKey   0x000f17       data     extern D:\Projects\PIC18_USB_Eval\Firmware\SoftPowerOnOff\SoftPowerOnOff\MainDemo.c
             KeyScanState   0x000f15       data     extern D:\Projects\PIC18_USB_Eval\Firmware\SoftPowerOnOff\SoftPowerOnOff\MainDemo.c
                     LATA   0x000f89       data     extern C:\MCC18\src\traditional\proc\p18F67J50.asm
                 LATAbits   0x000f89       data     extern C:\MCC18\src\traditional\proc\p18F67J50.asm
                     LATB   0x000f8a       data     extern C:\MCC18\src\traditional\proc\p18F67J50.asm
                 LATBbits   0x000f8a       data     extern C:\MCC18\src\traditional\proc\p18F67J50.asm
                     LATC   0x000f8b       data     extern C:\MCC18\src\traditional\proc\p18F67J50.asm
                 LATCbits   0x000f8b       data     extern C:\MCC18\src\traditional\proc\p18F67J50.asm
                     LATD   0x000f8c       data     extern C:\MCC18\src\traditional\proc\p18F67J50.asm
                 LATDbits   0x000f8c       data     extern C:\MCC18\src\traditional\proc\p18F67J50.asm
                     LATE   0x000f8d       data     extern C:\MCC18\src\traditional\proc\p18F67J50.asm
                 LATEbits   0x000f8d       data     extern C:\MCC18\src\traditional\proc\p18F67J50.asm
                     LATF   0x000f8e       data     extern C:\MCC18\src\traditional\proc\p18F67J50.asm
                 LATFbits   0x000f8e       data     extern C:\MCC18\src\traditional\proc\p18F67J50.asm
                     LATG   0x000f8f       data     extern C:\MCC18\src\traditional\proc\p18F67J50.asm
                 LATGbits   0x000f8f       data     extern C:\MCC18\src\traditional\proc\p18F67J50.asm
                 LEDState   0x000f14       data     extern D:\Projects\PIC18_USB_Eval\Firmware\SoftPowerOnOff\SoftPowerOnOff\MainDemo.c
                 MCUState   0x000f12       data     extern D:\Projects\PIC18_USB_Eval\Firmware\SoftPowerOnOff\SoftPowerOnOff\MainDemo.c
             MCUStateSave   0x000f13       data     extern D:\Projects\PIC18_USB_Eval\Firmware\SoftPowerOnOff\SoftPowerOnOff\MainDemo.c
                   ODCON1   0x000fcf       data     extern C:\MCC18\src\traditional\proc\p18F67J50.asm
               ODCON1bits   0x000fcf       data     extern C:\MCC18\src\traditional\proc\p18F67J50.asm
                   ODCON2   0x000fce       data     extern C:\MCC18\src\traditional\proc\p18F67J50.asm
               ODCON2bits   0x000fce       data     extern C:\MCC18\src\traditional\proc\p18F67J50.asm
                   ODCON3   0x000fcd       data     extern C:\MCC18\src\traditional\proc\p18F67J50.asm
               ODCON3bits   0x000fcd       data     extern C:\MCC18\src\traditional\proc\p18F67J50.asm
                   OSCCON   0x000fd3       data     extern C:\MCC18\src\traditional\proc\p18F67J50.asm
               OSCCONbits   0x000fd3       data     extern C:\MCC18\src\traditional\proc\p18F67J50.asm
                  OSCTUNE   0x000f9b       data     extern C:\MCC18\src\traditional\proc\p18F67J50.asm
              OSCTUNEbits   0x000f9b       data     extern C:\MCC18\src\traditional\proc\p18F67J50.asm
                  PADCFG1   0x000fcc       data     extern C:\MCC18\src\traditional\proc\p18F67J50.asm
              PADCFG1bits   0x000fcc       data     extern C:\MCC18\src\traditional\proc\p18F67J50.asm
                       PC   0x000ff9       data     extern C:\MCC18\src\traditional\proc\p18F67J50.asm
                      PCL   0x000ff9       data     extern C:\MCC18\src\traditional\proc\p18F67J50.asm
                   PCLATH   0x000ffa       data     extern C:\MCC18\src\traditional\proc\p18F67J50.asm
                   PCLATU   0x000ffb       data     extern C:\MCC18\src\traditional\proc\p18F67J50.asm
                     PIE1   0x000f9d       data     extern C:\MCC18\src\traditional\proc\p18F67J50.asm
                 PIE1bits   0x000f9d       data     extern C:\MCC18\src\traditional\proc\p18F67J50.asm
                     PIE2   0x000fa0       data     extern C:\MCC18\src\traditional\proc\p18F67J50.asm
                 PIE2bits   0x000fa0       data     extern C:\MCC18\src\traditional\proc\p18F67J50.asm
                     PIE3   0x000fa3       data     extern C:\MCC18\src\traditional\proc\p18F67J50.asm
                 PIE3bits   0x000fa3       data     extern C:\MCC18\src\traditional\proc\p18F67J50.asm
                     PIR1   0x000f9e       data     extern C:\MCC18\src\traditional\proc\p18F67J50.asm
                 PIR1bits   0x000f9e       data     extern C:\MCC18\src\traditional\proc\p18F67J50.asm
                     PIR2   0x000fa1       data     extern C:\MCC18\src\traditional\proc\p18F67J50.asm
                 PIR2bits   0x000fa1       data     extern C:\MCC18\src\traditional\proc\p18F67J50.asm
                     PIR3   0x000fa4       data     extern C:\MCC18\src\traditional\proc\p18F67J50.asm
                 PIR3bits   0x000fa4       data     extern C:\MCC18\src\traditional\proc\p18F67J50.asm
                   PLUSW0   0x000feb       data     extern C:\MCC18\src\traditional\proc\p18F67J50.asm
                   PLUSW1   0x000fe3       data     extern C:\MCC18\src\traditional\proc\p18F67J50.asm
                   PLUSW2   0x000fdb       data     extern C:\MCC18\src\traditional\proc\p18F67J50.asm
                   PMADDR   0x000f68       data     extern C:\MCC18\src\traditional\proc\p18F67J50.asm
                  PMADDRH   0x000f69       data     extern C:\MCC18\src\traditional\proc\p18F67J50.asm
              PMADDRHbits   0x000f69       data     extern C:\MCC18\src\traditional\proc\p18F67J50.asm
                  PMADDRL   0x000f68       data     extern C:\MCC18\src\traditional\proc\p18F67J50.asm
                    PMCON   0x000f4a       data     extern C:\MCC18\src\traditional\proc\p18F67J50.asm
                   PMCONH   0x000f4b       data     extern C:\MCC18\src\traditional\proc\p18F67J50.asm
               PMCONHbits   0x000f4b       data     extern C:\MCC18\src\traditional\proc\p18F67J50.asm
                   PMCONL   0x000f4a       data     extern C:\MCC18\src\traditional\proc\p18F67J50.asm
               PMCONLbits   0x000f4a       data     extern C:\MCC18\src\traditional\proc\p18F67J50.asm
                   PMDIN1   0x000f66       data     extern C:\MCC18\src\traditional\proc\p18F67J50.asm
                  PMDIN1H   0x000f67       data     extern C:\MCC18\src\traditional\proc\p18F67J50.asm
                  PMDIN1L   0x000f66       data     extern C:\MCC18\src\traditional\proc\p18F67J50.asm
                   PMDIN2   0x000f44       data     extern C:\MCC18\src\traditional\proc\p18F67J50.asm
                  PMDIN2H   0x000f45       data     extern C:\MCC18\src\traditional\proc\p18F67J50.asm
                  PMDIN2L   0x000f44       data     extern C:\MCC18\src\traditional\proc\p18F67J50.asm
                  PMDOUT1   0x000f68       data     extern C:\MCC18\src\traditional\proc\p18F67J50.asm
                 PMDOUT1H   0x000f69       data     extern C:\MCC18\src\traditional\proc\p18F67J50.asm
                 PMDOUT1L   0x000f68       data     extern C:\MCC18\src\traditional\proc\p18F67J50.asm
                  PMDOUT2   0x000f46       data     extern C:\MCC18\src\traditional\proc\p18F67J50.asm
                 PMDOUT2H   0x000f47       data     extern C:\MCC18\src\traditional\proc\p18F67J50.asm
                 PMDOUT2L   0x000f46       data     extern C:\MCC18\src\traditional\proc\p18F67J50.asm
                     PMEH   0x000f43       data     extern C:\MCC18\src\traditional\proc\p18F67J50.asm
                 PMEHbits   0x000f43       data     extern C:\MCC18\src\traditional\proc\p18F67J50.asm
                     PMEL   0x000f42       data     extern C:\MCC18\src\traditional\proc\p18F67J50.asm
                 PMELbits   0x000f42       data     extern C:\MCC18\src\traditional\proc\p18F67J50.asm
                     PMEN   0x000f42       data     extern C:\MCC18\src\traditional\proc\p18F67J50.asm
                   PMMODE   0x000f48       data     extern C:\MCC18\src\traditional\proc\p18F67J50.asm
                  PMMODEH   0x000f49       data     extern C:\MCC18\src\traditional\proc\p18F67J50.asm
              PMMODEHbits   0x000f49       data     extern C:\MCC18\src\traditional\proc\p18F67J50.asm
                  PMMODEL   0x000f48       data     extern C:\MCC18\src\traditional\proc\p18F67J50.asm
              PMMODELbits   0x000f48       data     extern C:\MCC18\src\traditional\proc\p18F67J50.asm
                   PMSTAT   0x000f40       data     extern C:\MCC18\src\traditional\proc\p18F67J50.asm
                  PMSTATH   0x000f41       data     extern C:\MCC18\src\traditional\proc\p18F67J50.asm
              PMSTATHbits   0x000f41       data     extern C:\MCC18\src\traditional\proc\p18F67J50.asm
                  PMSTATL   0x000f40       data     extern C:\MCC18\src\traditional\proc\p18F67J50.asm
              PMSTATLbits   0x000f40       data     extern C:\MCC18\src\traditional\proc\p18F67J50.asm
                    PORTA   0x000f80       data     extern C:\MCC18\src\traditional\proc\p18F67J50.asm
                PORTAbits   0x000f80       data     extern C:\MCC18\src\traditional\proc\p18F67J50.asm
                    PORTB   0x000f81       data     extern C:\MCC18\src\traditional\proc\p18F67J50.asm
                PORTBbits   0x000f81       data     extern C:\MCC18\src\traditional\proc\p18F67J50.asm
                    PORTC   0x000f82       data     extern C:\MCC18\src\traditional\proc\p18F67J50.asm
                PORTCbits   0x000f82       data     extern C:\MCC18\src\traditional\proc\p18F67J50.asm
                    PORTD   0x000f83       data     extern C:\MCC18\src\traditional\proc\p18F67J50.asm
                PORTDbits   0x000f83       data     extern C:\MCC18\src\traditional\proc\p18F67J50.asm
                    PORTE   0x000f84       data     extern C:\MCC18\src\traditional\proc\p18F67J50.asm
                PORTEbits   0x000f84       data     extern C:\MCC18\src\traditional\proc\p18F67J50.asm
                    PORTF   0x000f85       data     extern C:\MCC18\src\traditional\proc\p18F67J50.asm
                PORTFbits   0x000f85       data     extern C:\MCC18\src\traditional\proc\p18F67J50.asm
                    PORTG   0x000f86       data     extern C:\MCC18\src\traditional\proc\p18F67J50.asm
                PORTGbits   0x000f86       data     extern C:\MCC18\src\traditional\proc\p18F67J50.asm
                 POSTDEC0   0x000fed       data     extern C:\MCC18\src\traditional\proc\p18F67J50.asm
                 POSTDEC1   0x000fe5       data     extern C:\MCC18\src\traditional\proc\p18F67J50.asm
                 POSTDEC2   0x000fdd       data     extern C:\MCC18\src\traditional\proc\p18F67J50.asm
                 POSTINC0   0x000fee       data     extern C:\MCC18\src\traditional\proc\p18F67J50.asm
                 POSTINC1   0x000fe6       data     extern C:\MCC18\src\traditional\proc\p18F67J50.asm
                 POSTINC2   0x000fde       data     extern C:\MCC18\src\traditional\proc\p18F67J50.asm
                      PR2   0x000fcb       data     extern C:\MCC18\src\traditional\proc\p18F67J50.asm
                      PR4   0x000f77       data     extern C:\MCC18\src\traditional\proc\p18F67J50.asm
                  PREINC0   0x000fec       data     extern C:\MCC18\src\traditional\proc\p18F67J50.asm
                  PREINC1   0x000fe4       data     extern C:\MCC18\src\traditional\proc\p18F67J50.asm
                  PREINC2   0x000fdc       data     extern C:\MCC18\src\traditional\proc\p18F67J50.asm
                     PROD   0x000ff3       data     extern C:\MCC18\src\traditional\proc\p18F67J50.asm
                    PRODH   0x000ff4       data     extern C:\MCC18\src\traditional\proc\p18F67J50.asm
                    PRODL   0x000ff3       data     extern C:\MCC18\src\traditional\proc\p18F67J50.asm
                     RCON   0x000fd0       data     extern C:\MCC18\src\traditional\proc\p18F67J50.asm
                 RCONbits   0x000fd0       data     extern C:\MCC18\src\traditional\proc\p18F67J50.asm
                    RCREG   0x000faf       data     extern C:\MCC18\src\traditional\proc\p18F67J50.asm
                   RCREG1   0x000faf       data     extern C:\MCC18\src\traditional\proc\p18F67J50.asm
                   RCREG2   0x000faa       data     extern C:\MCC18\src\traditional\proc\p18F67J50.asm
                    RCSTA   0x000fac       data     extern C:\MCC18\src\traditional\proc\p18F67J50.asm
                   RCSTA1   0x000fac       data     extern C:\MCC18\src\traditional\proc\p18F67J50.asm
               RCSTA1bits   0x000fac       data     extern C:\MCC18\src\traditional\proc\p18F67J50.asm
                   RCSTA2   0x000f9c       data     extern C:\MCC18\src\traditional\proc\p18F67J50.asm
               RCSTA2bits   0x000f9c       data     extern C:\MCC18\src\traditional\proc\p18F67J50.asm
                RCSTAbits   0x000fac       data     extern C:\MCC18\src\traditional\proc\p18F67J50.asm
                  REFOCON   0x000fd3       data     extern C:\MCC18\src\traditional\proc\p18F67J50.asm
              REFOCONbits   0x000fd3       data     extern C:\MCC18\src\traditional\proc\p18F67J50.asm
                     SIGN   0x00000e       data     extern C:\MCC18\src\traditional\math\cmath18.asm
                    SPBRG   0x000fb0       data     extern C:\MCC18\src\traditional\proc\p18F67J50.asm
                   SPBRG1   0x000fb0       data     extern C:\MCC18\src\traditional\proc\p18F67J50.asm
                   SPBRG2   0x000fab       data     extern C:\MCC18\src\traditional\proc\p18F67J50.asm
                   SPBRGH   0x000f7f       data     extern C:\MCC18\src\traditional\proc\p18F67J50.asm
                  SPBRGH1   0x000f7f       data     extern C:\MCC18\src\traditional\proc\p18F67J50.asm
                  SPBRGH2   0x000f7d       data     extern C:\MCC18\src\traditional\proc\p18F67J50.asm
                  SSP1ADD   0x000fc8       data     extern C:\MCC18\src\traditional\proc\p18F67J50.asm
                  SSP1BUF   0x000fc9       data     extern C:\MCC18\src\traditional\proc\p18F67J50.asm
                 SSP1CON1   0x000fc6       data     extern C:\MCC18\src\traditional\proc\p18F67J50.asm
             SSP1CON1bits   0x000fc6       data     extern C:\MCC18\src\traditional\proc\p18F67J50.asm
                 SSP1CON2   0x000fc5       data     extern C:\MCC18\src\traditional\proc\p18F67J50.asm
             SSP1CON2bits   0x000fc5       data     extern C:\MCC18\src\traditional\proc\p18F67J50.asm
                  SSP1MSK   0x000fc8       data     extern C:\MCC18\src\traditional\proc\p18F67J50.asm
                 SSP1STAT   0x000fc7       data     extern C:\MCC18\src\traditional\proc\p18F67J50.asm
             SSP1STATbits   0x000fc7       data     extern C:\MCC18\src\traditional\proc\p18F67J50.asm
                  SSP2ADD   0x000f6e       data     extern C:\MCC18\src\traditional\proc\p18F67J50.asm
                  SSP2BUF   0x000f6f       data     extern C:\MCC18\src\traditional\proc\p18F67J50.asm
                 SSP2CON1   0x000f6c       data     extern C:\MCC18\src\traditional\proc\p18F67J50.asm
             SSP2CON1bits   0x000f6c       data     extern C:\MCC18\src\traditional\proc\p18F67J50.asm
                 SSP2CON2   0x000f6b       data     extern C:\MCC18\src\traditional\proc\p18F67J50.asm
             SSP2CON2bits   0x000f6b       data     extern C:\MCC18\src\traditional\proc\p18F67J50.asm
                  SSP2MSK   0x000f6e       data     extern C:\MCC18\src\traditional\proc\p18F67J50.asm
              SSP2MSKbits   0x000f6e       data     extern C:\MCC18\src\traditional\proc\p18F67J50.asm
                 SSP2STAT   0x000f6d       data     extern C:\MCC18\src\traditional\proc\p18F67J50.asm
             SSP2STATbits   0x000f6d       data     extern C:\MCC18\src\traditional\proc\p18F67J50.asm
                   SSPADD   0x000fc8       data     extern C:\MCC18\src\traditional\proc\p18F67J50.asm
                   SSPBUF   0x000fc9       data     extern C:\MCC18\src\traditional\proc\p18F67J50.asm
                  SSPCON1   0x000fc6       data     extern C:\MCC18\src\traditional\proc\p18F67J50.asm
              SSPCON1bits   0x000fc6       data     extern C:\MCC18\src\traditional\proc\p18F67J50.asm
                  SSPCON2   0x000fc5       data     extern C:\MCC18\src\traditional\proc\p18F67J50.asm
              SSPCON2bits   0x000fc5       data     extern C:\MCC18\src\traditional\proc\p18F67J50.asm
                  SSPSTAT   0x000fc7       data     extern C:\MCC18\src\traditional\proc\p18F67J50.asm
              SSPSTATbits   0x000fc7       data     extern C:\MCC18\src\traditional\proc\p18F67J50.asm
                   STATUS   0x000fd8       data     extern C:\MCC18\src\traditional\proc\p18F67J50.asm
               STATUSbits   0x000fd8       data     extern C:\MCC18\src\traditional\proc\p18F67J50.asm
                   STKPTR   0x000ffc       data     extern C:\MCC18\src\traditional\proc\p18F67J50.asm
               STKPTRbits   0x000ffc       data     extern C:\MCC18\src\traditional\proc\p18F67J50.asm
                    T0CON   0x000fd5       data     extern C:\MCC18\src\traditional\proc\p18F67J50.asm
                T0CONbits   0x000fd5       data     extern C:\MCC18\src\traditional\proc\p18F67J50.asm
                    T1CON   0x000fcd       data     extern C:\MCC18\src\traditional\proc\p18F67J50.asm
                T1CONbits   0x000fcd       data     extern C:\MCC18\src\traditional\proc\p18F67J50.asm
                    T2CON   0x000fca       data     extern C:\MCC18\src\traditional\proc\p18F67J50.asm
                T2CONbits   0x000fca       data     extern C:\MCC18\src\traditional\proc\p18F67J50.asm
                    T3CON   0x000f79       data     extern C:\MCC18\src\traditional\proc\p18F67J50.asm
                T3CONbits   0x000f79       data     extern C:\MCC18\src\traditional\proc\p18F67J50.asm
                    T4CON   0x000f76       data     extern C:\MCC18\src\traditional\proc\p18F67J50.asm
                T4CONbits   0x000f76       data     extern C:\MCC18\src\traditional\proc\p18F67J50.asm
                   TABLAT   0x000ff5       data     extern C:\MCC18\src\traditional\proc\p18F67J50.asm
                   TBLPTR   0x000ff6       data     extern C:\MCC18\src\traditional\proc\p18F67J50.asm
                  TBLPTRH   0x000ff7       data     extern C:\MCC18\src\traditional\proc\p18F67J50.asm
                  TBLPTRL   0x000ff6       data     extern C:\MCC18\src\traditional\proc\p18F67J50.asm
                  TBLPTRU   0x000ff8       data     extern C:\MCC18\src\traditional\proc\p18F67J50.asm
                    TMR0H   0x000fd7       data     extern C:\MCC18\src\traditional\proc\p18F67J50.asm
                    TMR0L   0x000fd6       data     extern C:\MCC18\src\traditional\proc\p18F67J50.asm
                    TMR1H   0x000fcf       data     extern C:\MCC18\src\traditional\proc\p18F67J50.asm
                    TMR1L   0x000fce       data     extern C:\MCC18\src\traditional\proc\p18F67J50.asm
                     TMR2   0x000fcc       data     extern C:\MCC18\src\traditional\proc\p18F67J50.asm
                    TMR3H   0x000f7b       data     extern C:\MCC18\src\traditional\proc\p18F67J50.asm
                    TMR3L   0x000f7a       data     extern C:\MCC18\src\traditional\proc\p18F67J50.asm
                     TMR4   0x000f78       data     extern C:\MCC18\src\traditional\proc\p18F67J50.asm
                      TOS   0x000ffd       data     extern C:\MCC18\src\traditional\proc\p18F67J50.asm
                     TOSH   0x000ffe       data     extern C:\MCC18\src\traditional\proc\p18F67J50.asm
                     TOSL   0x000ffd       data     extern C:\MCC18\src\traditional\proc\p18F67J50.asm
                     TOSU   0x000fff       data     extern C:\MCC18\src\traditional\proc\p18F67J50.asm
                    TRISA   0x000f92       data     extern C:\MCC18\src\traditional\proc\p18F67J50.asm
                TRISAbits   0x000f92       data     extern C:\MCC18\src\traditional\proc\p18F67J50.asm
                    TRISB   0x000f93       data     extern C:\MCC18\src\traditional\proc\p18F67J50.asm
                TRISBbits   0x000f93       data     extern C:\MCC18\src\traditional\proc\p18F67J50.asm
                    TRISC   0x000f94       data     extern C:\MCC18\src\traditional\proc\p18F67J50.asm
                TRISCbits   0x000f94       data     extern C:\MCC18\src\traditional\proc\p18F67J50.asm
                    TRISD   0x000f95       data     extern C:\MCC18\src\traditional\proc\p18F67J50.asm
                TRISDbits   0x000f95       data     extern C:\MCC18\src\traditional\proc\p18F67J50.asm
                    TRISE   0x000f96       data     extern C:\MCC18\src\traditional\proc\p18F67J50.asm
                TRISEbits   0x000f96       data     extern C:\MCC18\src\traditional\proc\p18F67J50.asm
                    TRISF   0x000f97       data     extern C:\MCC18\src\traditional\proc\p18F67J50.asm
                TRISFbits   0x000f97       data     extern C:\MCC18\src\traditional\proc\p18F67J50.asm
                    TRISG   0x000f98       data     extern C:\MCC18\src\traditional\proc\p18F67J50.asm
                TRISGbits   0x000f98       data     extern C:\MCC18\src\traditional\proc\p18F67J50.asm
                    TXREG   0x000fae       data     extern C:\MCC18\src\traditional\proc\p18F67J50.asm
                   TXREG1   0x000fae       data     extern C:\MCC18\src\traditional\proc\p18F67J50.asm
                   TXREG2   0x000fa9       data     extern C:\MCC18\src\traditional\proc\p18F67J50.asm
                    TXSTA   0x000fad       data     extern C:\MCC18\src\traditional\proc\p18F67J50.asm
                   TXSTA1   0x000fad       data     extern C:\MCC18\src\traditional\proc\p18F67J50.asm
               TXSTA1bits   0x000fad       data     extern C:\MCC18\src\traditional\proc\p18F67J50.asm
                   TXSTA2   0x000fa8       data     extern C:\MCC18\src\traditional\proc\p18F67J50.asm
               TXSTA2bits   0x000fa8       data     extern C:\MCC18\src\traditional\proc\p18F67J50.asm
                TXSTAbits   0x000fad       data     extern C:\MCC18\src\traditional\proc\p18F67J50.asm
                TickCount   0x000f18       data     static D:\Projects\PIC18_USB_Eval\Firmware\SoftPowerOnOff\Tick\tick.c
                    UADDR   0x000f5e       data     extern C:\MCC18\src\traditional\proc\p18F67J50.asm
                UADDRbits   0x000f5e       data     extern C:\MCC18\src\traditional\proc\p18F67J50.asm
                     UCFG   0x000f5f       data     extern C:\MCC18\src\traditional\proc\p18F67J50.asm
                 UCFGbits   0x000f5f       data     extern C:\MCC18\src\traditional\proc\p18F67J50.asm
                     UCON   0x000f65       data     extern C:\MCC18\src\traditional\proc\p18F67J50.asm
                 UCONbits   0x000f65       data     extern C:\MCC18\src\traditional\proc\p18F67J50.asm
                     UEIE   0x000f5d       data     extern C:\MCC18\src\traditional\proc\p18F67J50.asm
                 UEIEbits   0x000f5d       data     extern C:\MCC18\src\traditional\proc\p18F67J50.asm
                     UEIR   0x000f63       data     extern C:\MCC18\src\traditional\proc\p18F67J50.asm
                 UEIRbits   0x000f63       data     extern C:\MCC18\src\traditional\proc\p18F67J50.asm
                     UEP0   0x000f4c       data     extern C:\MCC18\src\traditional\proc\p18F67J50.asm
                 UEP0bits   0x000f4c       data     extern C:\MCC18\src\traditional\proc\p18F67J50.asm
                     UEP1   0x000f4d       data     extern C:\MCC18\src\traditional\proc\p18F67J50.asm
                    UEP10   0x000f56       data     extern C:\MCC18\src\traditional\proc\p18F67J50.asm
                UEP10bits   0x000f56       data     extern C:\MCC18\src\traditional\proc\p18F67J50.asm
                    UEP11   0x000f57       data     extern C:\MCC18\src\traditional\proc\p18F67J50.asm
                UEP11bits   0x000f57       data     extern C:\MCC18\src\traditional\proc\p18F67J50.asm
                    UEP12   0x000f58       data     extern C:\MCC18\src\traditional\proc\p18F67J50.asm
                UEP12bits   0x000f58       data     extern C:\MCC18\src\traditional\proc\p18F67J50.asm
                    UEP13   0x000f59       data     extern C:\MCC18\src\traditional\proc\p18F67J50.asm
                UEP13bits   0x000f59       data     extern C:\MCC18\src\traditional\proc\p18F67J50.asm
                    UEP14   0x000f5a       data     extern C:\MCC18\src\traditional\proc\p18F67J50.asm
                UEP14bits   0x000f5a       data     extern C:\MCC18\src\traditional\proc\p18F67J50.asm
                    UEP15   0x000f5b       data     extern C:\MCC18\src\traditional\proc\p18F67J50.asm
                UEP15bits   0x000f5b       data     extern C:\MCC18\src\traditional\proc\p18F67J50.asm
                 UEP1bits   0x000f4d       data     extern C:\MCC18\src\traditional\proc\p18F67J50.asm
                     UEP2   0x000f4e       data     extern C:\MCC18\src\traditional\proc\p18F67J50.asm
                 UEP2bits   0x000f4e       data     extern C:\MCC18\src\traditional\proc\p18F67J50.asm
                     UEP3   0x000f4f       data     extern C:\MCC18\src\traditional\proc\p18F67J50.asm
                 UEP3bits   0x000f4f       data     extern C:\MCC18\src\traditional\proc\p18F67J50.asm
                     UEP4   0x000f50       data     extern C:\MCC18\src\traditional\proc\p18F67J50.asm
                 UEP4bits   0x000f50       data     extern C:\MCC18\src\traditional\proc\p18F67J50.asm
                     UEP5   0x000f51       data     extern C:\MCC18\src\traditional\proc\p18F67J50.asm
                 UEP5bits   0x000f51       data     extern C:\MCC18\src\traditional\proc\p18F67J50.asm
                     UEP6   0x000f52       data     extern C:\MCC18\src\traditional\proc\p18F67J50.asm
                 UEP6bits   0x000f52       data     extern C:\MCC18\src\traditional\proc\p18F67J50.asm
                     UEP7   0x000f53       data     extern C:\MCC18\src\traditional\proc\p18F67J50.asm
                 UEP7bits   0x000f53       data     extern C:\MCC18\src\traditional\proc\p18F67J50.asm
                     UEP8   0x000f54       data     extern C:\MCC18\src\traditional\proc\p18F67J50.asm
                 UEP8bits   0x000f54       data     extern C:\MCC18\src\traditional\proc\p18F67J50.asm
                     UEP9   0x000f55       data     extern C:\MCC18\src\traditional\proc\p18F67J50.asm
                 UEP9bits   0x000f55       data     extern C:\MCC18\src\traditional\proc\p18F67J50.asm
                     UFRM   0x000f60       data     extern C:\MCC18\src\traditional\proc\p18F67J50.asm
                    UFRMH   0x000f61       data     extern C:\MCC18\src\traditional\proc\p18F67J50.asm
                UFRMHbits   0x000f61       data     extern C:\MCC18\src\traditional\proc\p18F67J50.asm
                    UFRML   0x000f60       data     extern C:\MCC18\src\traditional\proc\p18F67J50.asm
                UFRMLbits   0x000f60       data     extern C:\MCC18\src\traditional\proc\p18F67J50.asm
                      UIE   0x000f5c       data     extern C:\MCC18\src\traditional\proc\p18F67J50.asm
                  UIEbits   0x000f5c       data     extern C:\MCC18\src\traditional\proc\p18F67J50.asm
                      UIR   0x000f62       data     extern C:\MCC18\src\traditional\proc\p18F67J50.asm
                  UIRbits   0x000f62       data     extern C:\MCC18\src\traditional\proc\p18F67J50.asm
                    USTAT   0x000f64       data     extern C:\MCC18\src\traditional\proc\p18F67J50.asm
                USTATbits   0x000f64       data     extern C:\MCC18\src\traditional\proc\p18F67J50.asm
                   WDTCON   0x000fc0       data     extern C:\MCC18\src\traditional\proc\p18F67J50.asm
               WDTCONbits   0x000fc0       data     extern C:\MCC18\src\traditional\proc\p18F67J50.asm
                     WREG   0x000fe8       data     extern C:\MCC18\src\traditional\proc\p18F67J50.asm
                 __AARGB0   0x000007       data     extern C:\MCC18\src\traditional\math\aarg.asm
                 __AARGB1   0x000006       data     extern C:\MCC18\src\traditional\math\aarg.asm
                 __AARGB2   0x000005       data     extern C:\MCC18\src\traditional\math\aarg.asm
                 __AARGB3   0x000004       data     extern C:\MCC18\src\traditional\math\aarg.asm
                 __AARGB4   0x000003       data     extern C:\MCC18\src\traditional\math\aarg.asm
                 __AARGB5   0x000002       data     extern C:\MCC18\src\traditional\math\aarg.asm
                 __AARGB6   0x000001       data     extern C:\MCC18\src\traditional\math\aarg.asm
                 __AARGB7   0x000000       data     extern C:\MCC18\src\traditional\math\aarg.asm
                   __AEXP   0x000008       data     extern C:\MCC18\src\traditional\math\aarg.asm
                 __BARGB0   0x00000c       data     extern C:\MCC18\src\traditional\math\barg.asm
                 __BARGB1   0x00000b       data     extern C:\MCC18\src\traditional\math\barg.asm
                 __BARGB2   0x00000a       data     extern C:\MCC18\src\traditional\math\barg.asm
                 __BARGB3   0x000009       data     extern C:\MCC18\src\traditional\math\barg.asm
                   __BEXP   0x00000d       data     extern C:\MCC18\src\traditional\math\barg.asm
                __FPFLAGS   0x00000f       data     extern C:\MCC18\src\traditional\math\cmath18.asm
            __FPFLAGSbits   0x00000f       data     extern C:\MCC18\src\traditional\math\cmath18.asm
                  __REMB0   0x000003       data     extern C:\MCC18\src\traditional\math\aarg.asm
                  __REMB1   0x000002       data     extern C:\MCC18\src\traditional\math\aarg.asm
                  __REMB2   0x000001       data     extern C:\MCC18\src\traditional\math\aarg.asm
                  __REMB3   0x000000       data     extern C:\MCC18\src\traditional\math\aarg.asm
                  __tmp_0   0x000010       data     static D:\Projects\PIC18_USB_Eval\Firmware\SoftPowerOnOff\TimeDelay\TimeDelay.c
                  __tmp_0   0x000010       data     static D:\Projects\PIC18_USB_Eval\Firmware\SoftPowerOnOff\SoftPowerOnOff\MainDemo.c
                curr_byte   0x000f03       data     static C:\MCC18\src\traditional\startup\c018i.c
               curr_entry   0x000f05       data     static C:\MCC18\src\traditional\startup\c018i.c
                 data_ptr   0x000f07       data     static C:\MCC18\src\traditional\startup\c018i.c
                     prom   0x000f00       data     static C:\MCC18\src\traditional\startup\c018i.c
                       t1   0x000f0a       data     extern D:\Projects\PIC18_USB_Eval\Firmware\SoftPowerOnOff\SoftPowerOnOff\MainDemo.c
                       t2   0x000f0e       data     extern D:\Projects\PIC18_USB_Eval\Firmware\SoftPowerOnOff\SoftPowerOnOff\MainDemo.c



                              Symbols - Sorted by Address
                     Name    Address   Location    Storage File                     
                ---------  ---------  ---------  --------- ---------                
                   _entry   0x000000    program     extern C:\MCC18\src\traditional\startup\c018i.c
       ___return_lbl00000   0x000004    program     static                          
                 High_ISR   0x000008    program     extern D:\Projects\PIC18_USB_Eval\Firmware\SoftPowerOnOff\SoftPowerOnOff\MainDemo.c
       ___return_lbl00003   0x00000c    program     static                          
                  Low_ISR   0x000018    program     extern D:\Projects\PIC18_USB_Eval\Firmware\SoftPowerOnOff\SoftPowerOnOff\MainDemo.c
       ___return_lbl00004   0x00001c    program     static                          
                   _reset   0x001000    program     extern D:\Projects\PIC18_USB_Eval\Firmware\SoftPowerOnOff\SoftPowerOnOff\MainDemo.c
       ___return_lbl00000   0x001004    program     static                          
        Remapped_High_ISR   0x001008    program     extern D:\Projects\PIC18_USB_Eval\Firmware\SoftPowerOnOff\SoftPowerOnOff\MainDemo.c
       ___return_lbl00001   0x00100c    program     static                          
         Remapped_Low_ISR   0x001018    program     extern D:\Projects\PIC18_USB_Eval\Firmware\SoftPowerOnOff\SoftPowerOnOff\MainDemo.c
       ___return_lbl00002   0x00101c    program     static                          
  YourHighPriorityISRCode   0x001044    program     extern D:\Projects\PIC18_USB_Eval\Firmware\SoftPowerOnOff\SoftPowerOnOff\MainDemo.c
   YourLowPriorityISRCode   0x001110    program     extern D:\Projects\PIC18_USB_Eval\Firmware\SoftPowerOnOff\SoftPowerOnOff\MainDemo.c
                     main   0x001136    program     extern D:\Projects\PIC18_USB_Eval\Firmware\SoftPowerOnOff\SoftPowerOnOff\MainDemo.c
                   uiTask   0x00115a    program     extern D:\Projects\PIC18_USB_Eval\Firmware\SoftPowerOnOff\SoftPowerOnOff\MainDemo.c
           ___if_lbl00016   0x00116a    program     static                          
               __tmplbl_0   0x00119e    program     static                          
       ___case_0_lbl00019   0x0011b2    program     static                          
           ___if_lbl00018   0x0011c0    program     static                          
       ___case_1_lbl00022   0x0011c2    program     static                          
         ___else_lbl00021   0x0011ce    program     static                          
           ___if_lbl00020   0x0011d2    program     static                          
       ___case_2_lbl00025   0x0011d4    program     static                          
         ___else_lbl00024   0x0011de    program     static                          
           ___if_lbl00023   0x0011e4    program     static                          
   ___switchexit_lbl00017   0x0011e4    program     static                          
           ___?:_lbl00027   0x001208    program     static                          
           ___?:_lbl00026   0x00120e    program     static                          
           ___if_lbl00028   0x001218    program     static                          
           ___if_lbl00029   0x001218    program     static                          
         ___else_lbl00033   0x00121a    program     static                          
           ___if_lbl00030   0x00122c    program     static                          
           ___if_lbl00034   0x001234    program     static                          
           ___if_lbl00032   0x001234    program     static                          
           ___if_lbl00031   0x001234    program     static                          
               __tmplbl_2   0x00123c    program     static                          
               __tmplbl_3   0x001242    program     static                          
               __tmplbl_1   0x00124a    program     static                          
         ___else_lbl00038   0x001252    program     static                          
           ___if_lbl00037   0x001256    program     static                          
       ___return_lbl00015   0x00126a    program     static                          
           ___if_lbl00039   0x00126a    program     static                          
                  ledTask   0x00126c    program     extern D:\Projects\PIC18_USB_Eval\Firmware\SoftPowerOnOff\SoftPowerOnOff\MainDemo.c
                Delay10us   0x0012c2    program     extern D:\Projects\PIC18_USB_Eval\Firmware\SoftPowerOnOff\TimeDelay\TimeDelay.c
         ___else_lbl00006   0x0012d2    program     static                          
               __tmplbl_0   0x001374    program     static                          
         ___else_lbl00004   0x001378    program     static                          
        ___while_lbl00001   0x001378    program     static                          
               __tmplbl_1   0x0013a6    program     static                          
       ___return_lbl00000   0x0013c4    program     static                          
           ___if_lbl00005   0x0013c4    program     static                          
           ___if_lbl00003   0x0013c4    program     static                          
        ___while_lbl00002   0x0013c4    program     static                          
                  DelayMs   0x0013d8    program     extern D:\Projects\PIC18_USB_Eval\Firmware\SoftPowerOnOff\TimeDelay\TimeDelay.c
               __tmplbl_2   0x001480    program     static                          
        ___while_lbl00008   0x001486    program     static                          
         ___else_lbl00011   0x001486    program     static                          
               __tmplbl_3   0x0014b4    program     static                          
        ___while_lbl00009   0x0014d2    program     static                          
       ___return_lbl00007   0x0014d2    program     static                          
           ___if_lbl00010   0x0014d2    program     static                          
                _do_cinit   0x0014e6    program     extern C:\MCC18\src\traditional\startup\c018i.c
                     test   0x001500    program     static                          
                copy_loop   0x001558    program     static                          
            copy_one_byte   0x00155e    program     static                          
             done_copying   0x00156c    program     static                          
                     done   0x001582    program     static                          
       ___return_lbl00002   0x001582    program     static                          
                  FXM3232   0x001584    program     extern C:\MCC18\src\traditional\math\fxm3232.c
       ___return_lbl00000   0x0015f2    program     static                          
                 TickInit   0x0015f4    program     extern D:\Projects\PIC18_USB_Eval\Firmware\SoftPowerOnOff\Tick\tick.c
                  TickGet   0x001606    program     extern D:\Projects\PIC18_USB_Eval\Firmware\SoftPowerOnOff\Tick\tick.c
               TickUpdate   0x001618    program     extern D:\Projects\PIC18_USB_Eval\Firmware\SoftPowerOnOff\Tick\tick.c
            __zero_memory   0x00162e    program     extern C:\MCC18\src\traditional\proc\p18F67J50.asm
                   loop_h   0x00163c    program     static C:\MCC18\src\traditional\proc\p18F67J50.asm
               zero_block   0x00163c    program     static C:\MCC18\src\traditional\proc\p18F67J50.asm
                compare_l   0x001644    program     static C:\MCC18\src\traditional\proc\p18F67J50.asm
                   loop_l   0x001646    program     static C:\MCC18\src\traditional\proc\p18F67J50.asm
                 _startup   0x00164e    program     extern C:\MCC18\src\traditional\startup\c018i.c
                     loop   0x00165e    program     static                          
       ___return_lbl00001   0x001668    program     static                          
                   __init   0x00166a    program     extern C:\MCC18\src\traditional\stdclib\__init.c
               __config_0   0x01fff8    program     static D:\Projects\PIC18_USB_Eval\Firmware\SoftPowerOnOff\SoftPowerOnOff\MainDemo.c
               __config_1   0x01fff9    program     static D:\Projects\PIC18_USB_Eval\Firmware\SoftPowerOnOff\SoftPowerOnOff\MainDemo.c
               __config_2   0x01fffa    program     static D:\Projects\PIC18_USB_Eval\Firmware\SoftPowerOnOff\SoftPowerOnOff\MainDemo.c
               __config_3   0x01fffb    program     static D:\Projects\PIC18_USB_Eval\Firmware\SoftPowerOnOff\SoftPowerOnOff\MainDemo.c
               __config_4   0x01fffd    program     static D:\Projects\PIC18_USB_Eval\Firmware\SoftPowerOnOff\SoftPowerOnOff\MainDemo.c
                 __AARGB7   0x000000       data     extern C:\MCC18\src\traditional\math\aarg.asm
                  __REMB3   0x000000       data     extern C:\MCC18\src\traditional\math\aarg.asm
                 __AARGB6   0x000001       data     extern C:\MCC18\src\traditional\math\aarg.asm
                  __REMB2   0x000001       data     extern C:\MCC18\src\traditional\math\aarg.asm
                 __AARGB5   0x000002       data     extern C:\MCC18\src\traditional\math\aarg.asm
                  __REMB1   0x000002       data     extern C:\MCC18\src\traditional\math\aarg.asm
                  __REMB0   0x000003       data     extern C:\MCC18\src\traditional\math\aarg.asm
                 __AARGB4   0x000003       data     extern C:\MCC18\src\traditional\math\aarg.asm
                 __AARGB3   0x000004       data     extern C:\MCC18\src\traditional\math\aarg.asm
                 __AARGB2   0x000005       data     extern C:\MCC18\src\traditional\math\aarg.asm
                 __AARGB1   0x000006       data     extern C:\MCC18\src\traditional\math\aarg.asm
                 __AARGB0   0x000007       data     extern C:\MCC18\src\traditional\math\aarg.asm
                   __AEXP   0x000008       data     extern C:\MCC18\src\traditional\math\aarg.asm
                 __BARGB3   0x000009       data     extern C:\MCC18\src\traditional\math\barg.asm
                 __BARGB2   0x00000a       data     extern C:\MCC18\src\traditional\math\barg.asm
                 __BARGB1   0x00000b       data     extern C:\MCC18\src\traditional\math\barg.asm
                 __BARGB0   0x00000c       data     extern C:\MCC18\src\traditional\math\barg.asm
                   __BEXP   0x00000d       data     extern C:\MCC18\src\traditional\math\barg.asm
                     SIGN   0x00000e       data     extern C:\MCC18\src\traditional\math\cmath18.asm
            __FPFLAGSbits   0x00000f       data     extern C:\MCC18\src\traditional\math\cmath18.asm
                __FPFLAGS   0x00000f       data     extern C:\MCC18\src\traditional\math\cmath18.asm
                  __tmp_0   0x000010       data     static D:\Projects\PIC18_USB_Eval\Firmware\SoftPowerOnOff\TimeDelay\TimeDelay.c
                  __tmp_0   0x000010       data     static D:\Projects\PIC18_USB_Eval\Firmware\SoftPowerOnOff\SoftPowerOnOff\MainDemo.c
                     prom   0x000f00       data     static C:\MCC18\src\traditional\startup\c018i.c
                curr_byte   0x000f03       data     static C:\MCC18\src\traditional\startup\c018i.c
               curr_entry   0x000f05       data     static C:\MCC18\src\traditional\startup\c018i.c
                 data_ptr   0x000f07       data     static C:\MCC18\src\traditional\startup\c018i.c
                       t1   0x000f0a       data     extern D:\Projects\PIC18_USB_Eval\Firmware\SoftPowerOnOff\SoftPowerOnOff\MainDemo.c
                       t2   0x000f0e       data     extern D:\Projects\PIC18_USB_Eval\Firmware\SoftPowerOnOff\SoftPowerOnOff\MainDemo.c
                 MCUState   0x000f12       data     extern D:\Projects\PIC18_USB_Eval\Firmware\SoftPowerOnOff\SoftPowerOnOff\MainDemo.c
             MCUStateSave   0x000f13       data     extern D:\Projects\PIC18_USB_Eval\Firmware\SoftPowerOnOff\SoftPowerOnOff\MainDemo.c
                 LEDState   0x000f14       data     extern D:\Projects\PIC18_USB_Eval\Firmware\SoftPowerOnOff\SoftPowerOnOff\MainDemo.c
             KeyScanState   0x000f15       data     extern D:\Projects\PIC18_USB_Eval\Firmware\SoftPowerOnOff\SoftPowerOnOff\MainDemo.c
               KeyDownTmr   0x000f16       data     extern D:\Projects\PIC18_USB_Eval\Firmware\SoftPowerOnOff\SoftPowerOnOff\MainDemo.c
                KeyHitKey   0x000f17       data     extern D:\Projects\PIC18_USB_Eval\Firmware\SoftPowerOnOff\SoftPowerOnOff\MainDemo.c
                TickCount   0x000f18       data     static D:\Projects\PIC18_USB_Eval\Firmware\SoftPowerOnOff\Tick\tick.c
                   PMSTAT   0x000f40       data     extern C:\MCC18\src\traditional\proc\p18F67J50.asm
                  PMSTATL   0x000f40       data     extern C:\MCC18\src\traditional\proc\p18F67J50.asm
              PMSTATLbits   0x000f40       data     extern C:\MCC18\src\traditional\proc\p18F67J50.asm
                  PMSTATH   0x000f41       data     extern C:\MCC18\src\traditional\proc\p18F67J50.asm
              PMSTATHbits   0x000f41       data     extern C:\MCC18\src\traditional\proc\p18F67J50.asm
                 PMELbits   0x000f42       data     extern C:\MCC18\src\traditional\proc\p18F67J50.asm
                     PMEN   0x000f42       data     extern C:\MCC18\src\traditional\proc\p18F67J50.asm
                     PMEL   0x000f42       data     extern C:\MCC18\src\traditional\proc\p18F67J50.asm
                 PMEHbits   0x000f43       data     extern C:\MCC18\src\traditional\proc\p18F67J50.asm
                     PMEH   0x000f43       data     extern C:\MCC18\src\traditional\proc\p18F67J50.asm
                   PMDIN2   0x000f44       data     extern C:\MCC18\src\traditional\proc\p18F67J50.asm
                  PMDIN2L   0x000f44       data     extern C:\MCC18\src\traditional\proc\p18F67J50.asm
                  PMDIN2H   0x000f45       data     extern C:\MCC18\src\traditional\proc\p18F67J50.asm
                 PMDOUT2L   0x000f46       data     extern C:\MCC18\src\traditional\proc\p18F67J50.asm
                  PMDOUT2   0x000f46       data     extern C:\MCC18\src\traditional\proc\p18F67J50.asm
                 PMDOUT2H   0x000f47       data     extern C:\MCC18\src\traditional\proc\p18F67J50.asm
              PMMODELbits   0x000f48       data     extern C:\MCC18\src\traditional\proc\p18F67J50.asm
                  PMMODEL   0x000f48       data     extern C:\MCC18\src\traditional\proc\p18F67J50.asm
                   PMMODE   0x000f48       data     extern C:\MCC18\src\traditional\proc\p18F67J50.asm
              PMMODEHbits   0x000f49       data     extern C:\MCC18\src\traditional\proc\p18F67J50.asm
                  PMMODEH   0x000f49       data     extern C:\MCC18\src\traditional\proc\p18F67J50.asm
                    PMCON   0x000f4a       data     extern C:\MCC18\src\traditional\proc\p18F67J50.asm
                   PMCONL   0x000f4a       data     extern C:\MCC18\src\traditional\proc\p18F67J50.asm
               PMCONLbits   0x000f4a       data     extern C:\MCC18\src\traditional\proc\p18F67J50.asm
               PMCONHbits   0x000f4b       data     extern C:\MCC18\src\traditional\proc\p18F67J50.asm
                   PMCONH   0x000f4b       data     extern C:\MCC18\src\traditional\proc\p18F67J50.asm
                     UEP0   0x000f4c       data     extern C:\MCC18\src\traditional\proc\p18F67J50.asm
                 UEP0bits   0x000f4c       data     extern C:\MCC18\src\traditional\proc\p18F67J50.asm
                 UEP1bits   0x000f4d       data     extern C:\MCC18\src\traditional\proc\p18F67J50.asm
                     UEP1   0x000f4d       data     extern C:\MCC18\src\traditional\proc\p18F67J50.asm
                 UEP2bits   0x000f4e       data     extern C:\MCC18\src\traditional\proc\p18F67J50.asm
                     UEP2   0x000f4e       data     extern C:\MCC18\src\traditional\proc\p18F67J50.asm
                 UEP3bits   0x000f4f       data     extern C:\MCC18\src\traditional\proc\p18F67J50.asm
                     UEP3   0x000f4f       data     extern C:\MCC18\src\traditional\proc\p18F67J50.asm
                 UEP4bits   0x000f50       data     extern C:\MCC18\src\traditional\proc\p18F67J50.asm
                     UEP4   0x000f50       data     extern C:\MCC18\src\traditional\proc\p18F67J50.asm
                 UEP5bits   0x000f51       data     extern C:\MCC18\src\traditional\proc\p18F67J50.asm
                     UEP5   0x000f51       data     extern C:\MCC18\src\traditional\proc\p18F67J50.asm
                 UEP6bits   0x000f52       data     extern C:\MCC18\src\traditional\proc\p18F67J50.asm
                     UEP6   0x000f52       data     extern C:\MCC18\src\traditional\proc\p18F67J50.asm
                 UEP7bits   0x000f53       data     extern C:\MCC18\src\traditional\proc\p18F67J50.asm
                     UEP7   0x000f53       data     extern C:\MCC18\src\traditional\proc\p18F67J50.asm
                     UEP8   0x000f54       data     extern C:\MCC18\src\traditional\proc\p18F67J50.asm
                 UEP8bits   0x000f54       data     extern C:\MCC18\src\traditional\proc\p18F67J50.asm
                 UEP9bits   0x000f55       data     extern C:\MCC18\src\traditional\proc\p18F67J50.asm
                     UEP9   0x000f55       data     extern C:\MCC18\src\traditional\proc\p18F67J50.asm
                    UEP10   0x000f56       data     extern C:\MCC18\src\traditional\proc\p18F67J50.asm
                UEP10bits   0x000f56       data     extern C:\MCC18\src\traditional\proc\p18F67J50.asm
                    UEP11   0x000f57       data     extern C:\MCC18\src\traditional\proc\p18F67J50.asm
                UEP11bits   0x000f57       data     extern C:\MCC18\src\traditional\proc\p18F67J50.asm
                    UEP12   0x000f58       data     extern C:\MCC18\src\traditional\proc\p18F67J50.asm
                UEP12bits   0x000f58       data     extern C:\MCC18\src\traditional\proc\p18F67J50.asm
                    UEP13   0x000f59       data     extern C:\MCC18\src\traditional\proc\p18F67J50.asm
                UEP13bits   0x000f59       data     extern C:\MCC18\src\traditional\proc\p18F67J50.asm
                    UEP14   0x000f5a       data     extern C:\MCC18\src\traditional\proc\p18F67J50.asm
                UEP14bits   0x000f5a       data     extern C:\MCC18\src\traditional\proc\p18F67J50.asm
                    UEP15   0x000f5b       data     extern C:\MCC18\src\traditional\proc\p18F67J50.asm
                UEP15bits   0x000f5b       data     extern C:\MCC18\src\traditional\proc\p18F67J50.asm
                  UIEbits   0x000f5c       data     extern C:\MCC18\src\traditional\proc\p18F67J50.asm
                      UIE   0x000f5c       data     extern C:\MCC18\src\traditional\proc\p18F67J50.asm
                     UEIE   0x000f5d       data     extern C:\MCC18\src\traditional\proc\p18F67J50.asm
                 UEIEbits   0x000f5d       data     extern C:\MCC18\src\traditional\proc\p18F67J50.asm
                UADDRbits   0x000f5e       data     extern C:\MCC18\src\traditional\proc\p18F67J50.asm
                    UADDR   0x000f5e       data     extern C:\MCC18\src\traditional\proc\p18F67J50.asm
                 UCFGbits   0x000f5f       data     extern C:\MCC18\src\traditional\proc\p18F67J50.asm
                     UCFG   0x000f5f       data     extern C:\MCC18\src\traditional\proc\p18F67J50.asm
                UFRMLbits   0x000f60       data     extern C:\MCC18\src\traditional\proc\p18F67J50.asm
                    UFRML   0x000f60       data     extern C:\MCC18\src\traditional\proc\p18F67J50.asm
                     UFRM   0x000f60       data     extern C:\MCC18\src\traditional\proc\p18F67J50.asm
                UFRMHbits   0x000f61       data     extern C:\MCC18\src\traditional\proc\p18F67J50.asm
                    UFRMH   0x000f61       data     extern C:\MCC18\src\traditional\proc\p18F67J50.asm
                  UIRbits   0x000f62       data     extern C:\MCC18\src\traditional\proc\p18F67J50.asm
                      UIR   0x000f62       data     extern C:\MCC18\src\traditional\proc\p18F67J50.asm
                 UEIRbits   0x000f63       data     extern C:\MCC18\src\traditional\proc\p18F67J50.asm
                     UEIR   0x000f63       data     extern C:\MCC18\src\traditional\proc\p18F67J50.asm
                USTATbits   0x000f64       data     extern C:\MCC18\src\traditional\proc\p18F67J50.asm
                    USTAT   0x000f64       data     extern C:\MCC18\src\traditional\proc\p18F67J50.asm
                 UCONbits   0x000f65       data     extern C:\MCC18\src\traditional\proc\p18F67J50.asm
                     UCON   0x000f65       data     extern C:\MCC18\src\traditional\proc\p18F67J50.asm
                   PMDIN1   0x000f66       data     extern C:\MCC18\src\traditional\proc\p18F67J50.asm
                  PMDIN1L   0x000f66       data     extern C:\MCC18\src\traditional\proc\p18F67J50.asm
                  PMDIN1H   0x000f67       data     extern C:\MCC18\src\traditional\proc\p18F67J50.asm
                  PMADDRL   0x000f68       data     extern C:\MCC18\src\traditional\proc\p18F67J50.asm
                   PMADDR   0x000f68       data     extern C:\MCC18\src\traditional\proc\p18F67J50.asm
                 PMDOUT1L   0x000f68       data     extern C:\MCC18\src\traditional\proc\p18F67J50.asm
                  PMDOUT1   0x000f68       data     extern C:\MCC18\src\traditional\proc\p18F67J50.asm
                 PMDOUT1H   0x000f69       data     extern C:\MCC18\src\traditional\proc\p18F67J50.asm
              PMADDRHbits   0x000f69       data     extern C:\MCC18\src\traditional\proc\p18F67J50.asm
                  PMADDRH   0x000f69       data     extern C:\MCC18\src\traditional\proc\p18F67J50.asm
                   CMSTAT   0x000f6a       data     extern C:\MCC18\src\traditional\proc\p18F67J50.asm
                 CMSTATUS   0x000f6a       data     extern C:\MCC18\src\traditional\proc\p18F67J50.asm
             CMSTATUSbits   0x000f6a       data     extern C:\MCC18\src\traditional\proc\p18F67J50.asm
               CMSTATbits   0x000f6a       data     extern C:\MCC18\src\traditional\proc\p18F67J50.asm
             SSP2CON2bits   0x000f6b       data     extern C:\MCC18\src\traditional\proc\p18F67J50.asm
                 SSP2CON2   0x000f6b       data     extern C:\MCC18\src\traditional\proc\p18F67J50.asm
             SSP2CON1bits   0x000f6c       data     extern C:\MCC18\src\traditional\proc\p18F67J50.asm
                 SSP2CON1   0x000f6c       data     extern C:\MCC18\src\traditional\proc\p18F67J50.asm
             SSP2STATbits   0x000f6d       data     extern C:\MCC18\src\traditional\proc\p18F67J50.asm
                 SSP2STAT   0x000f6d       data     extern C:\MCC18\src\traditional\proc\p18F67J50.asm
              SSP2MSKbits   0x000f6e       data     extern C:\MCC18\src\traditional\proc\p18F67J50.asm
                  SSP2MSK   0x000f6e       data     extern C:\MCC18\src\traditional\proc\p18F67J50.asm
                  SSP2ADD   0x000f6e       data     extern C:\MCC18\src\traditional\proc\p18F67J50.asm
                  SSP2BUF   0x000f6f       data     extern C:\MCC18\src\traditional\proc\p18F67J50.asm
                  CCP5CON   0x000f70       data     extern C:\MCC18\src\traditional\proc\p18F67J50.asm
              CCP5CONbits   0x000f70       data     extern C:\MCC18\src\traditional\proc\p18F67J50.asm
                   CCPR5L   0x000f71       data     extern C:\MCC18\src\traditional\proc\p18F67J50.asm
                    CCPR5   0x000f71       data     extern C:\MCC18\src\traditional\proc\p18F67J50.asm
                   CCPR5H   0x000f72       data     extern C:\MCC18\src\traditional\proc\p18F67J50.asm
              CCP4CONbits   0x000f73       data     extern C:\MCC18\src\traditional\proc\p18F67J50.asm
                  CCP4CON   0x000f73       data     extern C:\MCC18\src\traditional\proc\p18F67J50.asm
                   CCPR4L   0x000f74       data     extern C:\MCC18\src\traditional\proc\p18F67J50.asm
                    CCPR4   0x000f74       data     extern C:\MCC18\src\traditional\proc\p18F67J50.asm
                   CCPR4H   0x000f75       data     extern C:\MCC18\src\traditional\proc\p18F67J50.asm
                T4CONbits   0x000f76       data     extern C:\MCC18\src\traditional\proc\p18F67J50.asm
                    T4CON   0x000f76       data     extern C:\MCC18\src\traditional\proc\p18F67J50.asm
                   CVRCON   0x000f77       data     extern C:\MCC18\src\traditional\proc\p18F67J50.asm
               CVRCONbits   0x000f77       data     extern C:\MCC18\src\traditional\proc\p18F67J50.asm
                      PR4   0x000f77       data     extern C:\MCC18\src\traditional\proc\p18F67J50.asm
                     TMR4   0x000f78       data     extern C:\MCC18\src\traditional\proc\p18F67J50.asm
                T3CONbits   0x000f79       data     extern C:\MCC18\src\traditional\proc\p18F67J50.asm
                    T3CON   0x000f79       data     extern C:\MCC18\src\traditional\proc\p18F67J50.asm
                    TMR3L   0x000f7a       data     extern C:\MCC18\src\traditional\proc\p18F67J50.asm
                    TMR3H   0x000f7b       data     extern C:\MCC18\src\traditional\proc\p18F67J50.asm
                 BAUDCON2   0x000f7c       data     extern C:\MCC18\src\traditional\proc\p18F67J50.asm
             BAUDCON2bits   0x000f7c       data     extern C:\MCC18\src\traditional\proc\p18F67J50.asm
                  SPBRGH2   0x000f7d       data     extern C:\MCC18\src\traditional\proc\p18F67J50.asm
                  BAUDCON   0x000f7e       data     extern C:\MCC18\src\traditional\proc\p18F67J50.asm
                 BAUDCON1   0x000f7e       data     extern C:\MCC18\src\traditional\proc\p18F67J50.asm
             BAUDCON1bits   0x000f7e       data     extern C:\MCC18\src\traditional\proc\p18F67J50.asm
              BAUDCONbits   0x000f7e       data     extern C:\MCC18\src\traditional\proc\p18F67J50.asm
                  SPBRGH1   0x000f7f       data     extern C:\MCC18\src\traditional\proc\p18F67J50.asm
                   SPBRGH   0x000f7f       data     extern C:\MCC18\src\traditional\proc\p18F67J50.asm
                PORTAbits   0x000f80       data     extern C:\MCC18\src\traditional\proc\p18F67J50.asm
                    PORTA   0x000f80       data     extern C:\MCC18\src\traditional\proc\p18F67J50.asm
                PORTBbits   0x000f81       data     extern C:\MCC18\src\traditional\proc\p18F67J50.asm
                    PORTB   0x000f81       data     extern C:\MCC18\src\traditional\proc\p18F67J50.asm
                PORTCbits   0x000f82       data     extern C:\MCC18\src\traditional\proc\p18F67J50.asm
                    PORTC   0x000f82       data     extern C:\MCC18\src\traditional\proc\p18F67J50.asm
                PORTDbits   0x000f83       data     extern C:\MCC18\src\traditional\proc\p18F67J50.asm
                    PORTD   0x000f83       data     extern C:\MCC18\src\traditional\proc\p18F67J50.asm
                PORTEbits   0x000f84       data     extern C:\MCC18\src\traditional\proc\p18F67J50.asm
                    PORTE   0x000f84       data     extern C:\MCC18\src\traditional\proc\p18F67J50.asm
                PORTFbits   0x000f85       data     extern C:\MCC18\src\traditional\proc\p18F67J50.asm
                    PORTF   0x000f85       data     extern C:\MCC18\src\traditional\proc\p18F67J50.asm
                PORTGbits   0x000f86       data     extern C:\MCC18\src\traditional\proc\p18F67J50.asm
                    PORTG   0x000f86       data     extern C:\MCC18\src\traditional\proc\p18F67J50.asm
                     LATA   0x000f89       data     extern C:\MCC18\src\traditional\proc\p18F67J50.asm
                 LATAbits   0x000f89       data     extern C:\MCC18\src\traditional\proc\p18F67J50.asm
                     LATB   0x000f8a       data     extern C:\MCC18\src\traditional\proc\p18F67J50.asm
                 LATBbits   0x000f8a       data     extern C:\MCC18\src\traditional\proc\p18F67J50.asm
                     LATC   0x000f8b       data     extern C:\MCC18\src\traditional\proc\p18F67J50.asm
                 LATCbits   0x000f8b       data     extern C:\MCC18\src\traditional\proc\p18F67J50.asm
                 LATDbits   0x000f8c       data     extern C:\MCC18\src\traditional\proc\p18F67J50.asm
                     LATD   0x000f8c       data     extern C:\MCC18\src\traditional\proc\p18F67J50.asm
                 LATEbits   0x000f8d       data     extern C:\MCC18\src\traditional\proc\p18F67J50.asm
                     LATE   0x000f8d       data     extern C:\MCC18\src\traditional\proc\p18F67J50.asm
                 LATFbits   0x000f8e       data     extern C:\MCC18\src\traditional\proc\p18F67J50.asm
                     LATF   0x000f8e       data     extern C:\MCC18\src\traditional\proc\p18F67J50.asm
                     LATG   0x000f8f       data     extern C:\MCC18\src\traditional\proc\p18F67J50.asm
                 LATGbits   0x000f8f       data     extern C:\MCC18\src\traditional\proc\p18F67J50.asm
                    TRISA   0x000f92       data     extern C:\MCC18\src\traditional\proc\p18F67J50.asm
                TRISAbits   0x000f92       data     extern C:\MCC18\src\traditional\proc\p18F67J50.asm
                 DDRAbits   0x000f92       data     extern C:\MCC18\src\traditional\proc\p18F67J50.asm
                     DDRA   0x000f92       data     extern C:\MCC18\src\traditional\proc\p18F67J50.asm
                    TRISB   0x000f93       data     extern C:\MCC18\src\traditional\proc\p18F67J50.asm
                 DDRBbits   0x000f93       data     extern C:\MCC18\src\traditional\proc\p18F67J50.asm
                     DDRB   0x000f93       data     extern C:\MCC18\src\traditional\proc\p18F67J50.asm
                TRISBbits   0x000f93       data     extern C:\MCC18\src\traditional\proc\p18F67J50.asm
                 DDRCbits   0x000f94       data     extern C:\MCC18\src\traditional\proc\p18F67J50.asm
                     DDRC   0x000f94       data     extern C:\MCC18\src\traditional\proc\p18F67J50.asm
                    TRISC   0x000f94       data     extern C:\MCC18\src\traditional\proc\p18F67J50.asm
                TRISCbits   0x000f94       data     extern C:\MCC18\src\traditional\proc\p18F67J50.asm
                    TRISD   0x000f95       data     extern C:\MCC18\src\traditional\proc\p18F67J50.asm
                TRISDbits   0x000f95       data     extern C:\MCC18\src\traditional\proc\p18F67J50.asm
                     DDRD   0x000f95       data     extern C:\MCC18\src\traditional\proc\p18F67J50.asm
                 DDRDbits   0x000f95       data     extern C:\MCC18\src\traditional\proc\p18F67J50.asm
                    TRISE   0x000f96       data     extern C:\MCC18\src\traditional\proc\p18F67J50.asm
                TRISEbits   0x000f96       data     extern C:\MCC18\src\traditional\proc\p18F67J50.asm
                     DDRE   0x000f96       data     extern C:\MCC18\src\traditional\proc\p18F67J50.asm
                 DDREbits   0x000f96       data     extern C:\MCC18\src\traditional\proc\p18F67J50.asm
                     DDRF   0x000f97       data     extern C:\MCC18\src\traditional\proc\p18F67J50.asm
                    TRISF   0x000f97       data     extern C:\MCC18\src\traditional\proc\p18F67J50.asm
                TRISFbits   0x000f97       data     extern C:\MCC18\src\traditional\proc\p18F67J50.asm
                 DDRFbits   0x000f97       data     extern C:\MCC18\src\traditional\proc\p18F67J50.asm
                    TRISG   0x000f98       data     extern C:\MCC18\src\traditional\proc\p18F67J50.asm
                TRISGbits   0x000f98       data     extern C:\MCC18\src\traditional\proc\p18F67J50.asm
                     DDRG   0x000f98       data     extern C:\MCC18\src\traditional\proc\p18F67J50.asm
                 DDRGbits   0x000f98       data     extern C:\MCC18\src\traditional\proc\p18F67J50.asm
                  OSCTUNE   0x000f9b       data     extern C:\MCC18\src\traditional\proc\p18F67J50.asm
              OSCTUNEbits   0x000f9b       data     extern C:\MCC18\src\traditional\proc\p18F67J50.asm
               RCSTA2bits   0x000f9c       data     extern C:\MCC18\src\traditional\proc\p18F67J50.asm
                   RCSTA2   0x000f9c       data     extern C:\MCC18\src\traditional\proc\p18F67J50.asm
                 PIE1bits   0x000f9d       data     extern C:\MCC18\src\traditional\proc\p18F67J50.asm
                     PIE1   0x000f9d       data     extern C:\MCC18\src\traditional\proc\p18F67J50.asm
                 PIR1bits   0x000f9e       data     extern C:\MCC18\src\traditional\proc\p18F67J50.asm
                     PIR1   0x000f9e       data     extern C:\MCC18\src\traditional\proc\p18F67J50.asm
                     IPR1   0x000f9f       data     extern C:\MCC18\src\traditional\proc\p18F67J50.asm
                 IPR1bits   0x000f9f       data     extern C:\MCC18\src\traditional\proc\p18F67J50.asm
                 PIE2bits   0x000fa0       data     extern C:\MCC18\src\traditional\proc\p18F67J50.asm
                     PIE2   0x000fa0       data     extern C:\MCC18\src\traditional\proc\p18F67J50.asm
                     PIR2   0x000fa1       data     extern C:\MCC18\src\traditional\proc\p18F67J50.asm
                 PIR2bits   0x000fa1       data     extern C:\MCC18\src\traditional\proc\p18F67J50.asm
                 IPR2bits   0x000fa2       data     extern C:\MCC18\src\traditional\proc\p18F67J50.asm
                     IPR2   0x000fa2       data     extern C:\MCC18\src\traditional\proc\p18F67J50.asm
                     PIE3   0x000fa3       data     extern C:\MCC18\src\traditional\proc\p18F67J50.asm
                 PIE3bits   0x000fa3       data     extern C:\MCC18\src\traditional\proc\p18F67J50.asm
                     PIR3   0x000fa4       data     extern C:\MCC18\src\traditional\proc\p18F67J50.asm
                 PIR3bits   0x000fa4       data     extern C:\MCC18\src\traditional\proc\p18F67J50.asm
                 IPR3bits   0x000fa5       data     extern C:\MCC18\src\traditional\proc\p18F67J50.asm
                     IPR3   0x000fa5       data     extern C:\MCC18\src\traditional\proc\p18F67J50.asm
                   EECON1   0x000fa6       data     extern C:\MCC18\src\traditional\proc\p18F67J50.asm
               EECON1bits   0x000fa6       data     extern C:\MCC18\src\traditional\proc\p18F67J50.asm
                   EECON2   0x000fa7       data     extern C:\MCC18\src\traditional\proc\p18F67J50.asm
               TXSTA2bits   0x000fa8       data     extern C:\MCC18\src\traditional\proc\p18F67J50.asm
                   TXSTA2   0x000fa8       data     extern C:\MCC18\src\traditional\proc\p18F67J50.asm
                   TXREG2   0x000fa9       data     extern C:\MCC18\src\traditional\proc\p18F67J50.asm
                   RCREG2   0x000faa       data     extern C:\MCC18\src\traditional\proc\p18F67J50.asm
                   SPBRG2   0x000fab       data     extern C:\MCC18\src\traditional\proc\p18F67J50.asm
                    RCSTA   0x000fac       data     extern C:\MCC18\src\traditional\proc\p18F67J50.asm
                   RCSTA1   0x000fac       data     extern C:\MCC18\src\traditional\proc\p18F67J50.asm
               RCSTA1bits   0x000fac       data     extern C:\MCC18\src\traditional\proc\p18F67J50.asm
                RCSTAbits   0x000fac       data     extern C:\MCC18\src\traditional\proc\p18F67J50.asm
                TXSTAbits   0x000fad       data     extern C:\MCC18\src\traditional\proc\p18F67J50.asm
               TXSTA1bits   0x000fad       data     extern C:\MCC18\src\traditional\proc\p18F67J50.asm
                   TXSTA1   0x000fad       data     extern C:\MCC18\src\traditional\proc\p18F67J50.asm
                    TXSTA   0x000fad       data     extern C:\MCC18\src\traditional\proc\p18F67J50.asm
                    TXREG   0x000fae       data     extern C:\MCC18\src\traditional\proc\p18F67J50.asm
                   TXREG1   0x000fae       data     extern C:\MCC18\src\traditional\proc\p18F67J50.asm
                   RCREG1   0x000faf       data     extern C:\MCC18\src\traditional\proc\p18F67J50.asm
                    RCREG   0x000faf       data     extern C:\MCC18\src\traditional\proc\p18F67J50.asm
                    SPBRG   0x000fb0       data     extern C:\MCC18\src\traditional\proc\p18F67J50.asm
                   SPBRG1   0x000fb0       data     extern C:\MCC18\src\traditional\proc\p18F67J50.asm
             ECCP3CONbits   0x000fb1       data     extern C:\MCC18\src\traditional\proc\p18F67J50.asm
                 ECCP3CON   0x000fb1       data     extern C:\MCC18\src\traditional\proc\p18F67J50.asm
                  CCP3CON   0x000fb1       data     extern C:\MCC18\src\traditional\proc\p18F67J50.asm
              CCP3CONbits   0x000fb1       data     extern C:\MCC18\src\traditional\proc\p18F67J50.asm
                    CCPR3   0x000fb2       data     extern C:\MCC18\src\traditional\proc\p18F67J50.asm
                   CCPR3L   0x000fb2       data     extern C:\MCC18\src\traditional\proc\p18F67J50.asm
                   CCPR3H   0x000fb3       data     extern C:\MCC18\src\traditional\proc\p18F67J50.asm
                 ECCP3DEL   0x000fb4       data     extern C:\MCC18\src\traditional\proc\p18F67J50.asm
             ECCP3DELbits   0x000fb4       data     extern C:\MCC18\src\traditional\proc\p18F67J50.asm
              ECCP3ASbits   0x000fb5       data     extern C:\MCC18\src\traditional\proc\p18F67J50.asm
                  ECCP3AS   0x000fb5       data     extern C:\MCC18\src\traditional\proc\p18F67J50.asm
                 ECCP2CON   0x000fb6       data     extern C:\MCC18\src\traditional\proc\p18F67J50.asm
             ECCP2CONbits   0x000fb6       data     extern C:\MCC18\src\traditional\proc\p18F67J50.asm
                  CCP2CON   0x000fb6       data     extern C:\MCC18\src\traditional\proc\p18F67J50.asm
              CCP2CONbits   0x000fb6       data     extern C:\MCC18\src\traditional\proc\p18F67J50.asm
                    CCPR2   0x000fb7       data     extern C:\MCC18\src\traditional\proc\p18F67J50.asm
                   CCPR2L   0x000fb7       data     extern C:\MCC18\src\traditional\proc\p18F67J50.asm
                   CCPR2H   0x000fb8       data     extern C:\MCC18\src\traditional\proc\p18F67J50.asm
             ECCP2DELbits   0x000fb9       data     extern C:\MCC18\src\traditional\proc\p18F67J50.asm
                 ECCP2DEL   0x000fb9       data     extern C:\MCC18\src\traditional\proc\p18F67J50.asm
              ECCP2ASbits   0x000fba       data     extern C:\MCC18\src\traditional\proc\p18F67J50.asm
                  ECCP2AS   0x000fba       data     extern C:\MCC18\src\traditional\proc\p18F67J50.asm
              CCP1CONbits   0x000fbb       data     extern C:\MCC18\src\traditional\proc\p18F67J50.asm
                  CCP1CON   0x000fbb       data     extern C:\MCC18\src\traditional\proc\p18F67J50.asm
                 ECCP1CON   0x000fbb       data     extern C:\MCC18\src\traditional\proc\p18F67J50.asm
             ECCP1CONbits   0x000fbb       data     extern C:\MCC18\src\traditional\proc\p18F67J50.asm
                   CCPR1L   0x000fbc       data     extern C:\MCC18\src\traditional\proc\p18F67J50.asm
                    CCPR1   0x000fbc       data     extern C:\MCC18\src\traditional\proc\p18F67J50.asm
                   CCPR1H   0x000fbd       data     extern C:\MCC18\src\traditional\proc\p18F67J50.asm
                 ECCP1DEL   0x000fbe       data     extern C:\MCC18\src\traditional\proc\p18F67J50.asm
             ECCP1DELbits   0x000fbe       data     extern C:\MCC18\src\traditional\proc\p18F67J50.asm
              ECCP1ASbits   0x000fbf       data     extern C:\MCC18\src\traditional\proc\p18F67J50.asm
                  ECCP1AS   0x000fbf       data     extern C:\MCC18\src\traditional\proc\p18F67J50.asm
                   WDTCON   0x000fc0       data     extern C:\MCC18\src\traditional\proc\p18F67J50.asm
               WDTCONbits   0x000fc0       data     extern C:\MCC18\src\traditional\proc\p18F67J50.asm
               ANCON0bits   0x000fc1       data     extern C:\MCC18\src\traditional\proc\p18F67J50.asm
                   ANCON0   0x000fc1       data     extern C:\MCC18\src\traditional\proc\p18F67J50.asm
                   ADCON1   0x000fc1       data     extern C:\MCC18\src\traditional\proc\p18F67J50.asm
               ADCON1bits   0x000fc1       data     extern C:\MCC18\src\traditional\proc\p18F67J50.asm
                   ADCON0   0x000fc2       data     extern C:\MCC18\src\traditional\proc\p18F67J50.asm
               ADCON0bits   0x000fc2       data     extern C:\MCC18\src\traditional\proc\p18F67J50.asm
                   ANCON1   0x000fc2       data     extern C:\MCC18\src\traditional\proc\p18F67J50.asm
               ANCON1bits   0x000fc2       data     extern C:\MCC18\src\traditional\proc\p18F67J50.asm
                    ADRES   0x000fc3       data     extern C:\MCC18\src\traditional\proc\p18F67J50.asm
                   ADRESL   0x000fc3       data     extern C:\MCC18\src\traditional\proc\p18F67J50.asm
                   ADRESH   0x000fc4       data     extern C:\MCC18\src\traditional\proc\p18F67J50.asm
              SSPCON2bits   0x000fc5       data     extern C:\MCC18\src\traditional\proc\p18F67J50.asm
                  SSPCON2   0x000fc5       data     extern C:\MCC18\src\traditional\proc\p18F67J50.asm
             SSP1CON2bits   0x000fc5       data     extern C:\MCC18\src\traditional\proc\p18F67J50.asm
                 SSP1CON2   0x000fc5       data     extern C:\MCC18\src\traditional\proc\p18F67J50.asm
             SSP1CON1bits   0x000fc6       data     extern C:\MCC18\src\traditional\proc\p18F67J50.asm
                  SSPCON1   0x000fc6       data     extern C:\MCC18\src\traditional\proc\p18F67J50.asm
              SSPCON1bits   0x000fc6       data     extern C:\MCC18\src\traditional\proc\p18F67J50.asm
                 SSP1CON1   0x000fc6       data     extern C:\MCC18\src\traditional\proc\p18F67J50.asm
                 SSP1STAT   0x000fc7       data     extern C:\MCC18\src\traditional\proc\p18F67J50.asm
             SSP1STATbits   0x000fc7       data     extern C:\MCC18\src\traditional\proc\p18F67J50.asm
                  SSPSTAT   0x000fc7       data     extern C:\MCC18\src\traditional\proc\p18F67J50.asm
              SSPSTATbits   0x000fc7       data     extern C:\MCC18\src\traditional\proc\p18F67J50.asm
                  SSP1MSK   0x000fc8       data     extern C:\MCC18\src\traditional\proc\p18F67J50.asm
                   SSPADD   0x000fc8       data     extern C:\MCC18\src\traditional\proc\p18F67J50.asm
                  SSP1ADD   0x000fc8       data     extern C:\MCC18\src\traditional\proc\p18F67J50.asm
                  SSP1BUF   0x000fc9       data     extern C:\MCC18\src\traditional\proc\p18F67J50.asm
                   SSPBUF   0x000fc9       data     extern C:\MCC18\src\traditional\proc\p18F67J50.asm
                    T2CON   0x000fca       data     extern C:\MCC18\src\traditional\proc\p18F67J50.asm
                T2CONbits   0x000fca       data     extern C:\MCC18\src\traditional\proc\p18F67J50.asm
                      PR2   0x000fcb       data     extern C:\MCC18\src\traditional\proc\p18F67J50.asm
                     TMR2   0x000fcc       data     extern C:\MCC18\src\traditional\proc\p18F67J50.asm
              PADCFG1bits   0x000fcc       data     extern C:\MCC18\src\traditional\proc\p18F67J50.asm
                  PADCFG1   0x000fcc       data     extern C:\MCC18\src\traditional\proc\p18F67J50.asm
               ODCON3bits   0x000fcd       data     extern C:\MCC18\src\traditional\proc\p18F67J50.asm
                    T1CON   0x000fcd       data     extern C:\MCC18\src\traditional\proc\p18F67J50.asm
                T1CONbits   0x000fcd       data     extern C:\MCC18\src\traditional\proc\p18F67J50.asm
                   ODCON3   0x000fcd       data     extern C:\MCC18\src\traditional\proc\p18F67J50.asm
                    TMR1L   0x000fce       data     extern C:\MCC18\src\traditional\proc\p18F67J50.asm
                   ODCON2   0x000fce       data     extern C:\MCC18\src\traditional\proc\p18F67J50.asm
               ODCON2bits   0x000fce       data     extern C:\MCC18\src\traditional\proc\p18F67J50.asm
                   ODCON1   0x000fcf       data     extern C:\MCC18\src\traditional\proc\p18F67J50.asm
               ODCON1bits   0x000fcf       data     extern C:\MCC18\src\traditional\proc\p18F67J50.asm
                    TMR1H   0x000fcf       data     extern C:\MCC18\src\traditional\proc\p18F67J50.asm
                 RCONbits   0x000fd0       data     extern C:\MCC18\src\traditional\proc\p18F67J50.asm
                     RCON   0x000fd0       data     extern C:\MCC18\src\traditional\proc\p18F67J50.asm
                   CM2CON   0x000fd1       data     extern C:\MCC18\src\traditional\proc\p18F67J50.asm
                  CM2CON1   0x000fd1       data     extern C:\MCC18\src\traditional\proc\p18F67J50.asm
               CM2CONbits   0x000fd1       data     extern C:\MCC18\src\traditional\proc\p18F67J50.asm
              CM2CON1bits   0x000fd1       data     extern C:\MCC18\src\traditional\proc\p18F67J50.asm
                   CM1CON   0x000fd2       data     extern C:\MCC18\src\traditional\proc\p18F67J50.asm
               CM1CONbits   0x000fd2       data     extern C:\MCC18\src\traditional\proc\p18F67J50.asm
                  CM1CON1   0x000fd2       data     extern C:\MCC18\src\traditional\proc\p18F67J50.asm
              CM1CON1bits   0x000fd2       data     extern C:\MCC18\src\traditional\proc\p18F67J50.asm
                   OSCCON   0x000fd3       data     extern C:\MCC18\src\traditional\proc\p18F67J50.asm
               OSCCONbits   0x000fd3       data     extern C:\MCC18\src\traditional\proc\p18F67J50.asm
                  REFOCON   0x000fd3       data     extern C:\MCC18\src\traditional\proc\p18F67J50.asm
              REFOCONbits   0x000fd3       data     extern C:\MCC18\src\traditional\proc\p18F67J50.asm
                T0CONbits   0x000fd5       data     extern C:\MCC18\src\traditional\proc\p18F67J50.asm
                    T0CON   0x000fd5       data     extern C:\MCC18\src\traditional\proc\p18F67J50.asm
                    TMR0L   0x000fd6       data     extern C:\MCC18\src\traditional\proc\p18F67J50.asm
                    TMR0H   0x000fd7       data     extern C:\MCC18\src\traditional\proc\p18F67J50.asm
               STATUSbits   0x000fd8       data     extern C:\MCC18\src\traditional\proc\p18F67J50.asm
                   STATUS   0x000fd8       data     extern C:\MCC18\src\traditional\proc\p18F67J50.asm
                     FSR2   0x000fd9       data     extern C:\MCC18\src\traditional\proc\p18F67J50.asm
                    FSR2L   0x000fd9       data     extern C:\MCC18\src\traditional\proc\p18F67J50.asm
                    FSR2H   0x000fda       data     extern C:\MCC18\src\traditional\proc\p18F67J50.asm
                   PLUSW2   0x000fdb       data     extern C:\MCC18\src\traditional\proc\p18F67J50.asm
                  PREINC2   0x000fdc       data     extern C:\MCC18\src\traditional\proc\p18F67J50.asm
                 POSTDEC2   0x000fdd       data     extern C:\MCC18\src\traditional\proc\p18F67J50.asm
                 POSTINC2   0x000fde       data     extern C:\MCC18\src\traditional\proc\p18F67J50.asm
                    INDF2   0x000fdf       data     extern C:\MCC18\src\traditional\proc\p18F67J50.asm
                      BSR   0x000fe0       data     extern C:\MCC18\src\traditional\proc\p18F67J50.asm
                     FSR1   0x000fe1       data     extern C:\MCC18\src\traditional\proc\p18F67J50.asm
                    FSR1L   0x000fe1       data     extern C:\MCC18\src\traditional\proc\p18F67J50.asm
                    FSR1H   0x000fe2       data     extern C:\MCC18\src\traditional\proc\p18F67J50.asm
                   PLUSW1   0x000fe3       data     extern C:\MCC18\src\traditional\proc\p18F67J50.asm
                  PREINC1   0x000fe4       data     extern C:\MCC18\src\traditional\proc\p18F67J50.asm
                 POSTDEC1   0x000fe5       data     extern C:\MCC18\src\traditional\proc\p18F67J50.asm
                 POSTINC1   0x000fe6       data     extern C:\MCC18\src\traditional\proc\p18F67J50.asm
                    INDF1   0x000fe7       data     extern C:\MCC18\src\traditional\proc\p18F67J50.asm
                     WREG   0x000fe8       data     extern C:\MCC18\src\traditional\proc\p18F67J50.asm
                     FSR0   0x000fe9       data     extern C:\MCC18\src\traditional\proc\p18F67J50.asm
                    FSR0L   0x000fe9       data     extern C:\MCC18\src\traditional\proc\p18F67J50.asm
                    FSR0H   0x000fea       data     extern C:\MCC18\src\traditional\proc\p18F67J50.asm
                   PLUSW0   0x000feb       data     extern C:\MCC18\src\traditional\proc\p18F67J50.asm
                  PREINC0   0x000fec       data     extern C:\MCC18\src\traditional\proc\p18F67J50.asm
                 POSTDEC0   0x000fed       data     extern C:\MCC18\src\traditional\proc\p18F67J50.asm
                 POSTINC0   0x000fee       data     extern C:\MCC18\src\traditional\proc\p18F67J50.asm
                    INDF0   0x000fef       data     extern C:\MCC18\src\traditional\proc\p18F67J50.asm
                  INTCON3   0x000ff0       data     extern C:\MCC18\src\traditional\proc\p18F67J50.asm
              INTCON3bits   0x000ff0       data     extern C:\MCC18\src\traditional\proc\p18F67J50.asm
              INTCON2bits   0x000ff1       data     extern C:\MCC18\src\traditional\proc\p18F67J50.asm
                  INTCON2   0x000ff1       data     extern C:\MCC18\src\traditional\proc\p18F67J50.asm
                   INTCON   0x000ff2       data     extern C:\MCC18\src\traditional\proc\p18F67J50.asm
               INTCONbits   0x000ff2       data     extern C:\MCC18\src\traditional\proc\p18F67J50.asm
                    PRODL   0x000ff3       data     extern C:\MCC18\src\traditional\proc\p18F67J50.asm
                     PROD   0x000ff3       data     extern C:\MCC18\src\traditional\proc\p18F67J50.asm
                    PRODH   0x000ff4       data     extern C:\MCC18\src\traditional\proc\p18F67J50.asm
                   TABLAT   0x000ff5       data     extern C:\MCC18\src\traditional\proc\p18F67J50.asm
                   TBLPTR   0x000ff6       data     extern C:\MCC18\src\traditional\proc\p18F67J50.asm
                  TBLPTRL   0x000ff6       data     extern C:\MCC18\src\traditional\proc\p18F67J50.asm
                  TBLPTRH   0x000ff7       data     extern C:\MCC18\src\traditional\proc\p18F67J50.asm
                  TBLPTRU   0x000ff8       data     extern C:\MCC18\src\traditional\proc\p18F67J50.asm
                       PC   0x000ff9       data     extern C:\MCC18\src\traditional\proc\p18F67J50.asm
                      PCL   0x000ff9       data     extern C:\MCC18\src\traditional\proc\p18F67J50.asm
                   PCLATH   0x000ffa       data     extern C:\MCC18\src\traditional\proc\p18F67J50.asm
                   PCLATU   0x000ffb       data     extern C:\MCC18\src\traditional\proc\p18F67J50.asm
                   STKPTR   0x000ffc       data     extern C:\MCC18\src\traditional\proc\p18F67J50.asm
               STKPTRbits   0x000ffc       data     extern C:\MCC18\src\traditional\proc\p18F67J50.asm
                     TOSL   0x000ffd       data     extern C:\MCC18\src\traditional\proc\p18F67J50.asm
                      TOS   0x000ffd       data     extern C:\MCC18\src\traditional\proc\p18F67J50.asm
                     TOSH   0x000ffe       data     extern C:\MCC18\src\traditional\proc\p18F67J50.asm
                     TOSU   0x000fff       data     extern C:\MCC18\src\traditional\proc\p18F67J50.asm


